:020000040000FA
:100000000C9431030C9459030C9459030C949228CA
:100010000C9492280C9492280C9459030C94590334
:100020000C9459030C9459030C9459030C945903E0
:100030000C9459030C9459030C9459030C945903D0
:100040000C9448280C9459030C9416280C94F0270F
:100050000C9459030C9459030C9459030C945903B0
:100060000C940A290C9459034E414E494E49545957
:10007000494E46CDCCCC3D0AD7233C17B7D1387773
:10008000CC2B329595E6241FB14F0A000020410089
:1000900000C84200401C4620BCBE4CCA1B0E5AAED3
:1000A000C59D7400407A10F35A00A0724E180900E2
:1000B00010A5D4E80000E87648170000E40B5402CD
:1000C0000000CA9A3B000000E1F505000080969808
:1000D00000000040420F000000A086010000001058
:1000E0002700000000E8030000000064000000009A
:1000F000000A00000000000100000000002C76D87B
:1001000088DC674F0823DFC1DFAE59E1B1B796E560
:10011000E3E453C63AE651997696E8E6C28426EBC4
:10012000898C9B62ED407C6FFCEFBC9C9F40F2BAD7
:10013000A56FA5F490055A2AF75C936B6CF9676D6F
:10014000C11BFCE0E40D47FEF520E6B500D0ED90C4
:100150002E0300943577050080841E080000204E91
:100160000A000000C80C333333330F986E1283112A
:1001700041EF8D2114893BE65516CFFEE6DB18D101
:10018000844B381BF77C1D901DA4BBE424203284D3
:10019000725E228100C9F124ECA1E53D2701080D22
:1001A00000FE09016102CD207FFE0BFE09FE0D005D
:1001B00080321989808080808080800080284383FD
:1001C0009090901367874848FC48FC48481259892A
:1001D0002078A0A0702828F02012698944A4481033
:1001E0001020485488126787609090609488743813
:1001F0001383808080323989204040808080404055
:10020000202239898040402020204040801665858A
:100210004830FC30481455852020F82020114383B5
:10022000706080165181F821338340E04002798963
:1002300002020408102040808012698930488484BA
:1002400084848448301259892060A02020202020F6
:10025000F81269897884840408304080FC12698926
:10026000FC040810380404847812698908182848A6
:100270008888FC0808126989FC8080B8C40404845A
:100280007812698938408080B8C48484781269897A
:10029000FC0408101020204040126989788484846E
:1002A00078848484781269897884848C740404083E
:1002B0007021388840E040000040E040114888202C
:1002C0007020000070608022598908102040804012
:1002D000201008146484FC0000FC1259898040201E
:1002E0001008102040801269897884840408101056
:1002F00000101269897884849CA4AC948078126977
:10030000893048848484FC848484126989F08884D8
:1003100088F0888488F01269897884808080808061
:100320008478126989F088848484848488F01269CE
:1003300089FC808080F0808080FC126989FC80804C
:1003400080F08080808012698978848080809C849D
:100350008C7412698984848484FC84848484125912
:1003600089F820202020202020F81279893E0808D2
:10037000080808088870126989848890A0C0A09035
:1003800088841269898080808080808080FC0279E6
:10039000898282C6AA92928282821269898484C4E6
:1003A000A4948C8484841269897884848484848469
:1003B0008478126989F8848484F880808080116A46
:1003C0008A788484848484A4947804126989F88463
:1003D0008484F8A090888412698978848080780465
:1003E000048478027989FE10101010101010101279
:1003F000698984848484848484847802798982826B
:100400004444442828281002798982828282929268
:1004100092AA440279898282442810284482820266
:100420007989828244281010101010126989FC0406
:10043000081020408080FC224989F08080808080E4
:100440008080F00279898080402010080402021226
:100450004989F010101010101010F018538320501C
:1004600088017181FE3A2282804012668678047C7F
:10047000848C74126989808080B8C48484C4B81262
:100480006686788480808478126989040404748C78
:1004900084848C741266867884FC808478126989DE
:1004A00038444040F8404040401068887488887064
:1004B00080788478126989808080B8C48484848438
:1004C00012588820006020202020F8105A8A080046
:1004D00018080808088888701269898080808890C8
:1004E000E09088841259896020202020202020F864
:1004F000027686EC9292929282126686B8C48484C6
:100500008484126686788484848478106888B8C469
:1005100084C4B8808080106888748C848C740404CF
:1005200004126686B8444040404012668678846073
:100530001884781268884040F84040404438126679
:1005400086888888888874125686888888505020C3
:1005500002768682829292AA44126686844830305D
:1005600048841068888484848C7404847812668635
:10057000FC08102040FC22598938404020C020400F
:100580004038321989808080808080808080125934
:1005900089E010102018201010E018538348A8900C
:1005A000FFFFE0FFD1AFFF32FFD1FFFEFFE0FFD141
:1005B000AEFFD1FFFEFFE0FFD11000FFFEFFD0FF36
:1005C000E0FFC1FFD1AED580A81FD300408D14201D
:1005D00002A1C8DA0281CFD9F1DB402EA4A6AFFF79
:1005E000D0FFFE005EBCE2613FDD83C29C7E20A3A3
:1005F000FD1F41009D23BE46DB65F88C11AF32CA5A
:1006000057E97400000000240027002A00000000C1
:1006100008000201000003040700000000000000C1
:100620000000000000230026002900000000002533
:100630000028002B00040404040404040402020241
:100640000202020303030303030102040810204013
:100650008001020408102001020408102000352A3D
:10066000652F11241FBECFEFD8E0DEBFCDBF26E03F
:10067000A6E4B3E001C01D92A13CB207E1F713E08C
:10068000A0E0B1E0E2EBF2E702C005900D92A634E3
:10069000B107D9F713E0C0E3D3E004C02197FE010E
:1006A0000E941537CF32D107C9F70E941E2C0C9437
:1006B0004C390C940000089580E0089580918506DF
:1006C00090918606009739F120919806FC0121113E
:1006D00023C03596E491E0939906FC013C96E491A1
:1006E000E0939A0680919906082E000C990B2091B0
:1006F0009A06821B910927FD939520919B06203431
:1007000041F0829FC001112426E0969587952A9595
:10071000E1F780939C060895213039F43F96E491E7
:10072000E0939906FC017096DACF3D96E491E09350
:100730009906FC013E96D3CF089508950895AF928F
:10074000BF92CF92DF92EF92FF920F931F93CF93BE
:10075000DF936C017B018B01040F151FEB015E0120
:10076000AE18BF08C017D10759F06991D601ED91B5
:10077000FC910190F081E02DC6010995892B79F754
:10078000C501DF91CF911F910F91FF90EF90DF9006
:10079000CF90BF90AF900895CF93DF93FC01448139
:1007A0005581608171818AE095E00E949F03EC0190
:1007B00042E050E060E871E08AE095E00E949F032B
:1007C0008C0F9D1FDF91CF910895FC01538D448DB7
:1007D000252F30E0842F90E0821B930B541710F0EC
:1007E000CF96089501970895FC01918D828D9817F9
:1007F00061F0A28DAE0FBF2FB11D5D968C91928DD1
:100800009F5F9F73928F90E008958FEF9FEF089501
:10081000FC01918D828D981731F0828DE80FF11DCA
:10082000858D90E008958FEF9FEF0895FC01918DE5
:10083000228D892F90E0805C9F4F821B91098F73DE
:10084000992708958AE095E00E94160421E0892BFB
:1008500009F420E0822F089580E090E0892B29F0B0
:100860000E94220481110C9400000895FC01A48DC3
:10087000A80FB92FB11DA35ABF4F2C91848D90E0C2
:1008800001968F739927848FA689B7892C93A089A5
:10089000B1898C91837080648C93938D848D98132F
:1008A00006C00288F389E02D80818F7D80830895C2
:1008B000EF92FF920F931F93CF93DF93EC0181E0B0
:1008C000888F9B8D8C8D98131AC0E889F989808157
:1008D00085FF15C09FB7F894EE89FF896083E8898A
:1008E000F98980818370806480839FBF81E090E07C
:1008F000DF91CF911F910F91FF90EF900895F62E09
:100900000B8D10E00F5F1F4F0F731127E02E8C8DA2
:100910008E110CC00FB607FCFACFE889F9898081E7
:1009200085FFF5CFCE010E943604F1CFEB8DEC0FA1
:10093000FD2FF11DE35AFF4FF0829FB7F8940B8F04
:10094000EA89FB8980818062CFCFCF93DF93EC016E
:10095000888D8823B9F0AA89BB89E889F9898C91A7
:1009600085FD03C0808186FD0DC00FB607FCF7CF63
:100970008C9185FFF2CF808185FFEDCFCE010E9463
:100980003604E9CFDF91CF91089590E0FC01E35F59
:10099000F94F2491FC01E75BF94F3491FC01EB5CCA
:1009A000F94FE491EE23C9F0222339F0233001F10D
:1009B000A8F4213019F1223029F1F0E0EE0FFF1FE9
:1009C000E55DF94FA591B4918FB7F894EC91611161
:1009D00026C030953E233C938FBF08952730A9F061
:1009E0002830C9F0243049F7809180008F7D03C002
:1009F000809180008F7780938000DFCF84B58F77E0
:100A000084BDDBCF84B58F7DFBCF8091B0008F7725
:100A10008093B000D2CF8091B0008F7DF9CF3E2B74
:100A2000DACFCF93DF9390E0FC01E75BF94F24919D
:100A30008B5C994FFC0184918823D1F090E0880F62
:100A4000991FFC01ED5FF94FA591B491FC01E55DA3
:100A5000F94FC591D49161110EC09FB7F8948C9154
:100A6000E22FE0958E238C932881E223E8839FBFB9
:100A7000DF91CF9108958FB7F894EC91E22BEC932E
:100A80008FBFF6CF8E3008F08E5020910E0190E48B
:100A9000299F900111248770822B80937C00809184
:100AA0007A00806480937A0080917A0086FDFCCF82
:100AB000809178009091790008953FB7F8948091E3
:100AC000A2049091A304A091A404B091A50426B51A
:100AD000A89B05C02F3F19F00196A11DB11D3FBF76
:100AE000BA2FA92F982F8827BC01CD01620F711D45
:100AF000811D911D42E0660F771F881F991F4A953F
:100B0000D1F708958F929F92AF92BF92CF92DF92CA
:100B1000EF92FF926B017C010E945D054B015C012D
:100B2000C114D104E104F104B9F00E945D05681913
:100B300079098A099B09683E73408105910580F314
:100B400021E0C21AD108E108F10888EE880E83E09E
:100B5000981EA11CB11CE4CFFF90EF90DF90CF90C6
:100B6000BF90AF909F908F9008958F929F92AF9279
:100B7000BF92CF92DF92EF92FF920F931F93CF938A
:100B8000DF938AE0A82EB12CD0E0C0E0EE24EA94F6
:100B900093E0F92E88248A9423E0922ED12CC12C44
:100BA00010E000E08FE00E9442050817190790F15D
:100BB000C816D90608F46C018815990568F18E15D8
:100BC0009F0508F47C01C80FD91F65E070E080E044
:100BD00090E00E94820581E0A81AB10819F70C0D77
:100BE0001D1DCE01801B910B8E199F098819990933
:100BF00066E070E00E94AC36CB01DF91CF911F918F
:100C00000F91FF90EF90DF90CF90BF90AF909F90AB
:100C10008F9008958C01D0CF4C01D5CF2FB7F89489
:100C200060919E0470919F048091A0049091A10412
:100C30002FBF0895DC0180E0615090F09D919827CE
:100C4000E92FEF70F0E0ED51FA4F2491E92FE29592
:100C5000EF70F0E0ED50FA4FE491822F8E27ECCF49
:100C60000895DC012C911196ED91FC91F89481810D
:100C7000822B81839281322F30959323928387E058
:100C800090E00197F1F781818323818383E290E0F3
:100C90000197F1F790817894EFECF0E03197F1F75C
:100CA000922381E009F480E00895FC0190810180A5
:100CB000F281E02D292F209560FF14C0F8948281E5
:100CC000822382838181892B8183A3E2B0E0119703
:100CD000F1F78281982B9283789487ED90E00197C9
:100CE000F1F70895F8948281822382838181892B90
:100CF0008183AFEFB0E01197F1F78281982B928357
:100D000078948FE090E0EBCFDF92EF92FF920F9319
:100D10001F93CF93DF93EC01D62EE42E08E010E072
:100D2000FF24F39461E08D2D8F2109F460E0CE0162
:100D30000E945506FF0C01501109A1F7E11010C0E7
:100D4000F894E981FA819181888180958923818352
:100D5000E981FA81928188818095892382837894C0
:100D6000DF91CF911F910F91FF90EF90DF90089549
:100D7000EF92FF920F931F93CF93DF938C017B0130
:100D800040E065E50E948406E70188E0E80EF11C7A
:100D9000699140E0C8010E948406CE15DF05C1F7C5
:100DA000DF91CF911F910F91FF90EF900895FC017B
:100DB00090810180F281E02DF8948181292F209586
:100DC0008223818378943DE743E050E0315029F15C
:100DD000DA011197F1F780818923C1F3F8948281B8
:100DE000822382838181892B81837894ABE7B7E06A
:100DF0001197F1F7F894818182238183A3E1B1E017
:100E00001197F1F78081982381E009F080E07894D0
:100E1000E3E6F6E03197F1F7089580E008958F92C8
:100E20009F92AF92BF92CF92DF92EF92FF92CF93B9
:100E3000DF93EC018E819F810E94D70640E06CEC2D
:100E40008E819F810E948406488164E48E819F8107
:100E50000E9484068A81882371F1E981E9508EEE2F
:100E6000C82E82E0D82EE33038F4F0E0EE0FFF1FFA
:100E7000E85CFE4FC080D1808B81882339F1888166
:100E8000811124C00E940E064B015C010D2C000C48
:100E9000EE08FF088E819F810E943106813059F053
:100EA0000E940E066C197D098E099F096815790547
:100EB0008A059B0578F3DF91CF91FF90EF90DF904B
:100EC000CF90BF90AF909F908F900895B601DD0CAA
:100ED000880B990BDF91CF91FF90EF90DF90CF902F
:100EE000BF90AF909F908F900C9482056F927F92ED
:100EF0008F929F92AF92BF92CF92DF92EF92FF922A
:100F00000F931F93CF93DF93EC017B018A018E81B6
:100F10009F810E94D706811102C090E037C0B701BF
:100F20008E819F810E94B80640E06EEB8E819F818A
:100F30000E9484067801680189E0C80ED11CAE8049
:100F4000BF8088E0882E912C712C66246394C501A3
:100F50000E94310681117628660CE1E08E1A910814
:100F6000B1F7F70171927F01EC15FD0541F78E8114
:100F70009F810E94D706813081F668E0C8010E94F7
:100F80001A0691E0F80120852813C7CF892FDF9139
:100F9000CF911F910F91FF90EF90DF90CF90BF9076
:100FA000AF909F908F907F906F900895CF93DF9335
:100FB000CDB7DEB729970FB6F894DEBF0FBECDBF11
:100FC000AE014F5F5F4F0E947607882331F08D811D
:100FD0008F33A9F020F48F31A1F080E007C08F3566
:100FE00021F08F37D1F78CE001C08BE029960FB646
:100FF000F894DEBF0FBECDBFDF91CF9108958AE098
:10100000F5CF89E0F3CF1F93CF93DF93EC01162F39
:1010100060E0812F0E941105612F70E0FB01E75B0A
:10102000F94FE491E883FB01EB5CF94FE491F0E0C8
:10103000EE0FFF1FEF5DF94F859194919A8389839D
:101040001B861D861C861A86198618861F821E829C
:101050001D821C821B82DF91CF911F9108952091E8
:101060009B0430919C042817390771F490919A04DD
:1010700080919904981741F0E0919A04F0E0E75AC2
:10108000FB4F808190E008958FEF9FEF08950895C2
:10109000EF92FF920F931F93CF93DF93DC015C9647
:1010A000ED90FC905D97E114F10479F481E090E01B
:1010B00013969C938E93129790E080E0DF91CF91EE
:1010C0001F910F91FF90EF9008955196ED91FC9133
:1010D000529750968C915097982F90950FB75E9697
:1010E0002C915E97122F127021FD6095F89420814B
:1010F000112319F1282B2083E7012197F1F728E02C
:10110000462F50E0308160FF1AC0382B3083E70152
:101110002197F1F7BA0175956795215089F7112349
:1011200081F08081892380830FBF5C968D919C9193
:101130000197F1F781E090E0C1CF2923DCCF39237B
:10114000E5CF9081892BEFCF20919B0430919C04B7
:101150002817390771F48091990420919A0490E03E
:10116000805C9F4F821B910960E470E00E94C03652
:10117000089590E080E0089520919B0430919C04B4
:1011800028173907B9F490919A0480919904981717
:1011900089F0E0919A04F0E0E75AFB4F80812091BA
:1011A0009A0430E02F5F3F4F2F73332720939A0428
:1011B00090E008958FEF9FEF0895E0919B04F091E8
:1011C0009C04E817F90769F4A389B4899C9185897F
:1011D000809589238C9310929C0410929B0481E04B
:1011E000089580E0089520913604260F3327331F99
:1011F00021323105ECF42091E004FC0190E080E024
:10120000243069F082E00895A09136042191AC0168
:101210004A5E5B4FA40FB52FB11D2C930196861724
:1012200098F380913604680F6093360480E0089547
:1012300081E008951092E00481E08093DF04109231
:10124000BA0461E082E10E94C50461E083E10E948A
:10125000C504E9EBF0E080818E7F808380818D7F03
:10126000808388E48093B80085E48093BC0008956F
:10127000CF93DF9391E0909315048823B9F0C09148
:10128000B800D091BA008091BC008A7B8093BC00EA
:1012900060E082E10E94C50460E083E10E94C50431
:1012A0000E941A09D093BA00C093B800DF91CF9181
:1012B00008958F929F92AF92BF92CF92DF92EF925A
:1012C000FF920F931F93CF93DF93D0910905D132F3
:1012D00008F0D7C0182FC09108050E945D056B016A
:1012E0007C018091E00481116BC082E08093E00476
:1012F0001093DF048FEF8093DE041092DD04D0930F
:10130000DC04A8EEB4E0ECEBF4E080E0D81391C08C
:101310001092BB048091BB04CC0FC82BC093BB04BC
:101320008091BA04813009F088C01092BA040E94FA
:101330005D056B017C018091BB048093BB008091B3
:10134000E2049091E304A091E404B091E504892BB8
:101350008A2B8B2BA1F00E945D050091E204109175
:10136000E3042091E4043091E5046C197D098E09B1
:101370009F09061717072807390708F442C080910C
:10138000BC0083FDD8CF85EC8093BC000E945D0536
:101390006B017C018091E004823009F450C080919F
:1013A000DE048F3F09F46FC08091DE04803209F4BF
:1013B0006CC08091DE04803309F469C084E026C0EB
:1013C0008091E2049091E304A091E404B091E504DB
:1013D000892B8A2B8B2B09F484CF0E945D0580908A
:1013E000E2049090E304A090E404B090E5046C194A
:1013F0007D098E099F0986169706A806B90608F08A
:1014000070CF8091E1040E94380985E01092E704D2
:10141000109209051092E604DF91CF911F910F9170
:10142000FF90EF90DF90CF90BF90AF909F908F9004
:1014300008959D9191938F5F69CF85EEA5CF80919F
:10144000E2049091E304A091E404B091E504892BB7
:101450008A2B8B2B09F49ECF0E945D050091E2043C
:101460001091E3042091E4043091E5046C197D09A6
:101470008E099F09061717072807390708F08ACF32
:10148000C0CF81E0C3CF80E0C1CF82E0BFCF83E097
:10149000BDCFE091AB048091AA04E81730F4F0E0EE
:1014A000EB50FC4F808190E008958FEF9FEF0895FF
:1014B0009091AB048091AA042FEF3FEF981748F466
:1014C000E92FF0E0EB50FC4F208130E09F5F9093DC
:1014D000AB04C90108958091AA049091AB04891BC3
:1014E000990B0895CF92DF92EF92FF920F931F9383
:1014F000CF93DF937C01CB018A012091E604222364
:1015000089F0EB016B01C40ED51ECC15DD0569F029
:101510006991D701ED91FC910190F081E02DC70117
:101520000995F3CF642F0E94F308C801DF91CF9192
:101530001F910F91FF90EF90DF90CF900895CF9380
:10154000DF931F92CDB7DEB769832091E604222393
:10155000F9F020910905203258F021E030E0FC013B
:101560003383228390E080E00F90DF91CF91089544
:101570008091E704E82FF0E0E851FB4F99819083D8
:101580008F5F8093E7048093090581E090E0ECCFC2
:1015900061E0CE0101960E94F308F7CF80E0089544
:1015A000DC011696ED91FC91179712968C91481BD1
:1015B000477081E090E001C0880F4A95EAF7E60F96
:1015C000F11D3081222319F0832B808308958095AB
:1015D0008323FBCFFB014181DC0112962C911297F2
:1015E000421768F013962C911397241740F06081EE
:1015F00015962C91621718F424810C94D00A089542
:10160000FC0180819281980F92832181921760F46E
:1016100094819F5F94839381890F821710F08FEFDD
:10162000820F838381E0089580E00895FC01128297
:1016300080818150838314820895DB01ED91FC91B8
:101640000994CF93DF931F92CDB7DEB79E012F5F32
:101650003F4F47E40E941D0B89810F90DF91CF918E
:101660000895CF93DF931F92CDB7DEB79E012F5F12
:101670003F4F46E40E941D0B89810F90DF91CF916F
:101680000895BF92CF92DF92EF92FF920F931F9334
:10169000CF93DF938C01D42EE901FB01E280F3802C
:1016A000F2E34F1709F476C0F417C8F08CE248173C
:1016B00009F470C0EDE24E17E9F0F7E14F1779F148
:1016C0009E014D2DB701C801DF91CF911F910F9160
:1016D000FF90EF90DF90CF90BF900C941D0B86E4AD
:1016E000481709F44CC0E7E44E1709F44EC0FBE379
:1016F0004F13E6CFB701C8010E94210BC980C094E7
:10170000C80EB701C8010E94310B98819095890FCE
:101710008883C9828B818E5F83708B834BC047E146
:10172000B701C8010E941D0BB701C8010E94310B0F
:10173000BA80B094B80EB701C8010E94310BD880AE
:10174000D094D80EB701C8010E94210BCB80C09461
:10175000C80EB701C8010E94210B99819095890F8D
:10176000B882C982DA828B8381E0DF91CF911F91A9
:101770000F91FF90EF90DF90CF90BF900895B70149
:10178000C8010E94310B8883EFCFB701C8010E94C6
:10179000210BF9CFB701C8010E94210BC980C09469
:1017A000C80EB701C8010E94310B98819095890F2E
:1017B0008883C9829E014D2DB701C8010E941D0B6F
:1017C000D3CFCF93DF93EC016A817B810E94310BF1
:1017D00088836A817B81CE010E94210B89836A8183
:1017E0007B8130E020E048E4CE010E941D0B8B8716
:1017F0009E012D5C3F4F6A817B8147E1CE01DF91E5
:10180000CF910C941D0BCF93DF93C0918306D091A1
:101810008406E091B206F091B30682E0099530E0CB
:1018200020E04AE0BE0181E896E00E941D0BC82F2F
:10183000E091B206F091B30683E00995E091B2061B
:10184000F091B30680E00995CC2329F081E896E079
:101850000E94E10BC1E08C2FDF91CF910895FC0134
:10186000808D8F5F08950B96FC01849108950A96F0
:10187000FC0184910895FC01849108950E943B0C21
:10188000882321F0823011F083E0089586E00895E6
:10189000FC01E60FF11D849190E0982F8827319686
:1018A000E4918E0F911D089568E00C94480C66E059
:1018B0000C94480C5F926F927F928F929F92AF929E
:1018C000BF92CF92DF92EF92FF920F931F93CF932D
:1018D000DF93EC01E62EF42EC22E0C811D81C8018F
:1018E0000E943B0CD82E8C819D810E943E0C982E2C
:1018F00021E0AA24AA94D21202C02FE0A22E8C8149
:101900009D810E94370CD82E8C819D810E94330CC2
:10191000B82E8C819D810E94540CE0E6EC1578F481
:10192000009769F0080F191F91E6D92EBC14C0F476
:10193000188A1B8A1C8A198A1A8A80E0A0C08C81A6
:101940009D810E94570CF0E4FC1538F4009729F0B3
:10195000080F191F81E4D82EE9CF0F5E1F4FE6CF85
:10196000BD1430F3892D90E0F80124912F3F31F41C
:101970000F5F1F4FBD14E1F2D394F6CFCD1072C0AC
:101980008C819D810E943B0C98012F5F3F4FF80195
:10199000882319F0823009F04EC084918B8BF901B5
:1019A00024912C8BF8013396E491E88BF80134965E
:1019B000E491E98BF8013596E491EA8B0115110564
:1019C00009F4BBCF8C819D810E943E0C3C89F31AA7
:1019D0009A89F91A9FEF930F9F0D2CA94EA94F15C5
:1019E00008F449C0921718F49F1508F047C02B89D6
:1019F0009989E90E9FEF920F9E0D4BA95DA95E1587
:101A000008F44DC0941718F49E1508F037C0080F5D
:101A1000111D295F722E7694769476946F2C630E46
:101A20005E01FCE1AF0EB11C872C912CF61431F154
:101A30005E2C68014AC08491982F9F7092509A8BB7
:101A400082958F70898BF9012491822F8F708C8BF6
:101A500022952F702B8BF8013296E491E295EF706E
:101A6000E88BACCF3296E491EA21E80FF92FF11D13
:101A70000E0F1F1F7FCF921708F0B6CF8889DF9116
:101A8000CF911F910F91FF90EF90DF90CF90BF907B
:101A9000AF909F908F907F906F905F900895941774
:101AA00008F0B2CFEBCFF60184916A817B815C8E26
:101AB000FD8E1F8E8E8F95014BE3CE010E941D0B74
:101AC000FFEFCF1ADF0A28E0520E8C2D801B8715FE
:101AD00050F3080D191DF394A9CF2EE93FE00097AC
:101AE00009F40895F9013197F1F70197F8CFCF93F1
:101AF000DF9300D0CDB7DEB720ED37E03A832983FE
:101B00009091BC00982311F081E00FC029813A81A7
:101B1000232B81F48091B90481FDF6CF8091B80424
:101B200081110DC091E09093B8040F900F90DF9158
:101B3000CF91089529813A8121503109DFCF80E08A
:101B4000F4CF84EA8093BC0061E080E80E94770DC6
:101B5000811102C080E008958091B900887F8830AB
:101B600051F0803141F08091B8048111F3CF82E0CF
:101B70008093B804EFCF88E78093BB0084E880931C
:101B8000BC0062E080E80E94770D882319F3809101
:101B9000B90481FD05C08091B900887F883119F7AB
:101BA00081E0089584E98093BC0064E080E10C94B6
:101BB000770D8093BB0084E88093BC0063E080E8ED
:101BC0000E94770D8823A1F08091B90481FD0DC09A
:101BD0008091B900887F883241F08091B8048111EA
:101BE00006C092E09093B804089581E0089580E0E3
:101BF00008951092B80408958093B9041092B90022
:101C000088E48093B8000C94F90DCF93DF93FC0126
:101C100023A5222389F0EC010E94A10D811104C0AB
:101C200080E0DF91CF9108958EA1811107C00E94BD
:101C3000D90D8823A9F31BA681E0F3CF80E4F7CF69
:101C40000F931F93CF93DF93C62FD42F8901633057
:101C500001F138F4613099F0623009F449C0C1E013
:101C600012C0663029F1673091F16530C1F70E94EA
:101C7000050E811117C00E94D20DC0E004C0FC0106
:101C800086A50E94FC0D8C2FDF91CF911F910F91A3
:101C90000895FC0116A221E023A74111E0CF0E9484
:101CA000D20DDDCF8D2F0E94D90D8111D8CFE3CF7A
:101CB0000E94050E8823F9F2DD2389F2F801819153
:101CC0008F010E94D90D8823B1F2D150F5CF0E9427
:101CD000050E882381F2DD2311F2F80184910E9420
:101CE000D90DC82F882379F20F5F1F4FD150F3CF42
:101CF000FC0146A321E023A7B2CFDB011496ED91AE
:101D0000FC9130E020E065E00994CF92DF92EF9201
:101D1000FF920F931F93CF93DF938C017B016A0196
:101D200080E0F601C491811110C081E0CF3F49F0FD
:101D30004C2FB701C8010E947D0E882309F44DC0C5
:101D400080E0BFEFCB1ADB0AECCF4FEFCF3F89F338
:101D5000CE3F09F443C0C03F98F7C03E60F04C2F1F
:101D60004F70D7011496ED91FC9130E020E062E0D5
:101D7000C8010995E5CFC03D50F04C2F4F70D701F9
:101D80001496ED91FC9130E020E063E0F1CFC03C8F
:101D9000F8F0D7011496ED91FC9130E020E040E09E
:101DA00064E0C8010995C295C07FCE5FD0E0CE0146
:101DB0000E946D0DD7011496ED91FC9130E020E06A
:101DC00041E064E0C8010995CE010E946D0DB8CFD5
:101DD000C7FDB6CF8C2F90E0F8CF80E0DF91CF9198
:101DE0001F910F91FF90EF90DF90CF900895AF92E9
:101DF000BF92CF92DF92FF920F931F93CF93DF9307
:101E00006C018B01F42EE90180E1481709F484C0CC
:101E1000841758F1AAE04A1709F462C0F801028158
:101E20001381F2E3FF1609F4CDC0FF1508F47FC05B
:101E300085E1F81609F4CBC0A7E1FA1609F4DCC075
:101E4000B4E1FB126FC0D8011696ED91FC91179783
:101E500015968C918E0F9F2F911D11928E179F07B3
:101E6000E1F7C8010E94160B5DC0B1E14B1709F400
:101E70005BC0E5E14E13D2CFFB01A280B38045EBFE
:101E800055E0C6010E94850ED50114964C91406B19
:101E9000B801C6010E947D0ED8011496ED91FC9107
:101EA00030E020E041E062E0C6010995F5012681BD
:101EB0003781D8011496ED91FC91D50115964C917E
:101EC00066E0C601099581111CC080E0DF91CF91C9
:101ED0001F910F91FF90DF90CF90BF90AF9008952A
:101EE000DB011496ED91FC9130E020E042E061E0EE
:101EF000C60109954DEB55E0B801C6010E94850E5B
:101F00008DCFD8011496ED91FC9130E020E040E0B7
:101F100063E0C601099582CF4CEA55E0B801C601DD
:101F20000E94850E81E0D2CF41EA55E0F7CFE6E48A
:101F3000FE1609F46BC0F7E4FF1609F46CC08BE3DE
:101F4000F812F0CF99818B8138E0390F813031F070
:101F5000833011F0392F02C0392F985021E0D80179
:101F600013964C91491708F420E041E0391708F026
:101F700040E091E0F8015281351708F490E0322FEB
:101F8000342B932311F4242369F2FA80D12CC12C31
:101F9000843048F490E0FC01EC5CFE4FC080805D32
:101FA0009E4FDC01DC90F7FE04C0BE01C8010E9418
:101FB000EA0A88818C0D888389818D0D8983FF0CC5
:101FC00091F7B0CFBE01C8010E94EA0AABCFC801A9
:101FD0000E94000B882309F478CFD8011696ED9162
:101FE000FC91179715968C918E0F9F2F911D119232
:101FF0008E179F07E1F796CF1882F80182818983B7
:10200000858181508A8383818B838CCFD8011596FB
:102010008C91888387CFF8018181FBCF8EE596E094
:102020000E94DD08109279061092780610927706C9
:102030001092760610927506109274068DE991E062
:1020400090937B0680937A0690916A06963108F009
:1020500046C02DEB30E030937506209374062BE9D3
:1020600031E030937706209376062CE231E030930E
:102070007906209378062091680084E0983048F033
:1020800031E09E3008F430E081E001C0880F3A95DD
:10209000EAF7822B809368002DE630E0983050F00C
:1020A0002BE630E09E3030F02CE630E0963110F038
:1020B00030E020E03093720620937106292F30E043
:1020C0009830C0F581E001C0880F9A95EAF78093B7
:1020D000730680917A0690917B060197F1F78091C3
:1020E000780690917906892B21F180919B0490913B
:1020F0009C0426E08E359207E1F0009711F00E94D3
:10210000DD0880917C068E7F80937C061092990476
:1021100010929A048EE596E090939C0480939B0421
:10212000E0917106F0917206808190917306892B7F
:10213000808308959E3040F42850310981E001C029
:10214000880F2A95EAF7C3CF2E503109F7CF2F9287
:102150003F924F925F926F927F928F929F92AF9237
:10216000BF92CF92DF92EF92FF920F931F93CF9384
:10217000DF93CDB7DEB72D970FB6F894DEBF0FBE55
:10218000CDBF1C010E940E1064E670E080E090E07C
:102190000E9482056AE070E080E090E00E94820583
:1021A000C101880F991F9D878C87D12CC12CF12CE0
:1021B000E12C412C512C320149E050E067E271E002
:1021C0008EE596E00E949F0365E070E080E090E07D
:1021D0000E94820510E000E0812C912C54018EE5D4
:1021E00096E00E94A408892B39F4F4E08F1691043C
:1021F000A104B1040CF05FC0023011050CF05BC00B
:102200008EE596E00E94A408892B99F08EE596E071
:102210000E94BC08E1E0F0E0EC0FFD1FE00FF11FB1
:1022200080836AE070E080E090E00E9482050F5FAA
:102230001F4F65E070E080E090E00E948205023070
:10224000110509F070C089818F3F09F06CC08A8147
:10225000863809F068C0FE013396FB87EA878EE571
:1022600096E00E94A408892B39F4F4E08F169104BB
:10227000A104B1040CF050C00930110509F059C097
:102280008B8190E0982F88272C81820F911D092E39
:10229000000CAA0BBB0B480E591E6A1E7B1E40C0C9
:1022A000EC85FD85EC15FD0509F086CFE114F10400
:1022B00041F4710106C08FEFC81AD80AE214F30482
:1022C0007CF3C301B2010E9406344B015C01B701EB
:1022D000FF0C880B990B0E9406349B01AC01C501D1
:1022E000B4010E94FA352D960FB6F894DEBF0FBEEA
:1022F000CDBFDF91CF911F910F91FF90EF90DF90B5
:10230000CF90BF90AF909F908F907F906F905F9095
:102310004F903F902F900895043011050CF0B0CFEE
:10232000FFEFEF1AFF0A8FEF881A980AA80AB80A77
:1023300056CF8EE596E00E94BC08EA85FB85819326
:10234000FB87EA870F5F1F4F8ACFDF92EF92FF92E2
:102350000F931F93CF93DF93EC01D62E1CAD0BADE3
:102360007C0184E0E80EF11CE98DFA8DC701099526
:10237000412F480F2D2D602FC7010E945A0C9BAD95
:10238000890F8BAF81E090E0DF91CF911F910F918A
:10239000FF90EF90DF90089590E080E00895BF9265
:1023A000CF92DF92EF92FF920F931F93CF93DF9321
:1023B000EC01B62EC72E8D85811105C0CE010E947D
:1023C000D70681110EC01B861D861C8680E0DF911A
:1023D000CF911F910F91FF90EF90DF90CF90BF9022
:1023E000089540E060EFCE010E94840601E0E12CF8
:1023F000D12C11E0CE010E943106F82ECE010E94B0
:10240000310691E0F91218C0813099F51134D8F2F3
:10241000DB86D11002C081E08D878B81882399F201
:102420002396EB2DFC2DCF01089629912193E817D7
:10243000F907D9F781E0CBCFEE2DF0E0F8120FC00D
:102440008B851817A0F4DE01AE0FBF1F13968C9179
:10245000802379F4F12C193008F41C87D12EEC0F6D
:10246000FD1F8381902F9095892383830AC0811358
:10247000F1CFFE01EE0DF11D8381802B8383FF24BC
:10248000F3946F2DCE010E9455061F5F000F11F4CB
:10249000E39401E087E08E1508F0ACCFB7CFDF9270
:1024A000EF92FF920F931F93CF93DF937C018B01E9
:1024B000D42EDC011696ED91FC91138615861486B8
:1024C0001286118610861782168215821482138254
:1024D000C0E0B801F701868197810E94CF11D82F03
:1024E000882329F0DC1629F0CF5FDC1690F7D0E0C6
:1024F00009C067E0C8010E941A06D80117969C918E
:102500008913F2CF8D2FDF91CF911F910F91FF9003
:10251000EF90DF9008950F931F93CF93DF93CDB784
:10252000DEB761970FB6F894DEBF0FBECDBF8C014A
:10253000462FBE01665F7F4F0E944F1281110FC070
:1025400060E070E08EEF92EC61960FB6F894DEBF1B
:102550000FBECDBFDF91CF911F910F910895AE01B6
:102560004F5F5F4FBE01665F7F4FC8010E947607D5
:10257000882331F36A8170E0762F6627770F770F13
:10258000770F298148E0249F90011124262B372BB7
:102590008A858031D1F4688570E08F81AB01481B5A
:1025A0005109CA019695982F8827979587950E947B
:1025B000C036CB014097B90153E0660F771F5A959B
:1025C000E1F760789C01260F371F213854EE35075C
:1025D0000CF4B6CFB901330F880B990B0E94063467
:1025E00020E030E040E05CE30E946534ADCFEF9244
:1025F000FF920F931F93CF93DF93CDB7DEB728974A
:102600000FB6F894DEBF0FBECDBF8C01DC0116966D
:10261000ED91FC9117971386158614861286118604
:1026200010861782168215821482138214961C92C9
:10263000149715961C92EE24E394BE016F5F7F4FB2
:10264000F801868197810E94CF11882309F46FC019
:1026500067E0CE0101960E941A0698858913EDCF96
:10266000D8018C91811125C016968D919C910E9464
:10267000D706BE016F5F7F4FF801868197810E9468
:10268000B80640E064EBD80116968D919C910E94AB
:102690008406F801868197810E943106F82ED801C0
:1026A00016968D919C910E94D706F11002C0F801F8
:1026B000E082D8011196FC9089818031A1F1BE01A0
:1026C0006F5F7F4FC8010E94D6078F15D0F4F801C5
:1026D0008181D80111968C93119714968C9114973F
:1026E0008F5F14968C938981883231F0B0F48031F9
:1026F00019F0823209F0A1CFF80185818F5F8583BF
:102700009CCF8981803111F48CE0E3CFBE016F5FF3
:102710007F4FC8010E94D607DCCF8B3369F3823428
:1027200009F08BCFE9CFFCE0FF1588F2EDCF2896BA
:102730000FB6F894DEBF0FBECDBFDF91CF911F91D2
:102740000F91FF90EF9008959F92AF92BF92CF921A
:10275000DF92EF92FF920F931F93CF93DF93CDB74A
:10276000DEB761970FB6F894DEBF0FBECDBF8C0108
:102770008CE0F8018183D12CC12C2FE5E22E3FE7BC
:10278000B32E4FE1A42E5FE3952EF80184818C15C2
:102790001D0409F00CF4A3C04C2DBE01665F7F4FF1
:1027A000C8010E944F12F801F180FCE0FF1550F5BE
:1027B0009CE0F92E8A85803159F1BE01665F7F4F1A
:1027C000C8010E94D607F81609F481C0AE014F5F18
:1027D0005F4FBE01665F7F4FC8010E947607882366
:1027E00009F475C08A85803109F471C0EBE0FE16EA
:1027F00009F471C0FCE0FF1669F08AE0F8126DC0C0
:102800009D8209C089E0F816A8F689E0F82ED2CF9B
:102810008CE0D9CFBD82F801868197810E94D706CE
:10282000BE01665F7F4FF801868197810E94B806DE
:1028300040E06EE4F801868197810E94840640E0C2
:102840006B81F801868197810E94840640E06C814B
:10285000F801868197810E9484068A85803139F04B
:1028600040E06D81F801868197810E948406F8011D
:10287000868197810E94D706BE01665F7F4FF8016F
:10288000868197810E94B806F801408168E48681BC
:1028900097810E94840664E170E080E090E00E94ED
:1028A0008205F8018081882331F06AE070E080E0E1
:1028B00090E00E948205F801868197810E94D706E8
:1028C000F80181818F1508F48F2DF8018183FFEFC6
:1028D000CF1ADF0A5ACFED829ECFAD829CCF619690
:1028E0000FB6F894DEBF0FBECDBFDF91CF911F9121
:1028F0000F91FF90EF90DF90CF90BF90AF909F909F
:1029000008950F931F93CF93DF93FC0104811581EA
:102910000115110539F4FB011082DF91CF911F9150
:102920000F910895415051094017510708F48A0149
:10293000EB01FC0160817181A801CE010E94233965
:10294000C00FD11F1882E9CFCF93DF93C0915206F9
:10295000D0915306209761F08991882349F0082E81
:10296000000C990B0E94FD38FE0131978083F4CF53
:10297000DF91CF91089585ED8093BC008091E204B2
:102980009091E304A091E404B091E5040796A11DA1
:10299000B11D23E0B695A795979587952A95D1F710
:1029A0002091BC0024FD03C01092E00408954091E2
:1029B000E2045091E3046091E4047091E504452B36
:1029C000462B472B69F30097A105B10541F025E39C
:1029D0002A95F1F700000197A109B109E1CF809193
:1029E000E1040C943809FC0180819181009711F079
:1029F0000C94B52F60E070E0CB010895FB01448199
:102A00005581FC01248135812417350778F08081B8
:102A10009181009759F0FB01608171816115710509
:102A200029F00E94153921E0892B09F020E0822F3E
:102A300008950F931F93CF93DF938C01EB01FC015B
:102A4000808191810097E1F068817981611571053C
:102A5000A9F0428153812C813D814217530770F0C8
:102A60000E940E398C819D81F801958384831D829B
:102A70001C82DF91CF911F910F9108950E94B7376B
:102A800088819981F801918380838A819B819383D6
:102A900082838C819D8195838483198218821B8215
:102AA0001A82E5CFCF93DF93EC018881998100975B
:102AB00011F00E94B737198218821D821C821B8276
:102AC0001A82DF91CF910895FC0180819181009756
:102AD00011F00C94B73708950F931F93CF93DF93A2
:102AE000EC0188819981009759F02A813B81261752
:102AF000370730F081E0DF91CF911F910F9108955A
:102B00008B016F5F7F4F0E944038009759F0998387
:102B100088831B830A832C813D81232B59F7FC0179
:102B20001082E8CF80E0E7CFEF92FF920F931F93E0
:102B3000CF93DF936115710541F480E0DF91CF9170
:102B40001F910F91FF90EF90089541155105B1F03D
:102B50007B01EC010C811D81040F151FB8010E943F
:102B60006C15882351F3288139818C819D81B701AF
:102B7000820F931F0E940E391D830C8381E0DECFEC
:102B8000FC01448155816081718188E596E00C9457
:102B900094150F931F93CF93DF9300D0CDB7DEB77B
:102BA0008C0169831A8241E050E0BE016F5F7F4F64
:102BB0000E949415811103C0C8010E945215C801DA
:102BC0000F900F90DF91CF911F910F910895CF93A8
:102BD000DF93EC01FB0101900020E9F73197AF0191
:102BE000461B570B0E949415811103C0CE010E9411
:102BF0005215CE01DF91CF910895CF93DF93EC0171
:102C0000FB0144815581608171810E94941581117D
:102C100003C0CE010E945215CE01DF91CF910895DD
:102C2000EF92FF920F931F93CF93DF93EC017B0101
:102C30008A01BA010E946C1581110BC0CE010E945D
:102C40005215CE01DF91CF911F910F91FF90EF9020
:102C500008951D830C83B701888199810E940E39E4
:102C6000F0CFFB0101900020E9F73197AF01461B3F
:102C7000570B0C9410160F931F93CF93DF93CDB780
:102C8000DEB762970FB6F894DEBF0FBECDBF8C01E2
:102C9000CB01F801118210821382128215821482F4
:102CA0004AE0BE016F5F7F4F0E94DC2FBE016F5F65
:102CB0007F4FC8010E94311662960FB6F894DEBFAE
:102CC0000FBECDBFDF91CF911F910F910895CF938C
:102CD000DF93EC01FB018617970749F06081718152
:102CE0006115710541F0448155810E941016CE0195
:102CF000DF91CF9108950E945215F9CFFC01118206
:102D0000108213821282158214820C946716FC01C1
:102D1000118210821382128215821482611571054C
:102D200051F0FB0101900020E9F73197AF01461BFC
:102D3000570B0C9410160895AF92BF92CF92DF926A
:102D4000EF92FF920F931F93CF93DF936C015B0180
:102D50007A0189012417350720F48F2D7901042F7A
:102D6000182F62E871E0C6010E948716D5011496FB
:102D7000CD91DC91EC16FD06E0F40C171D0708F46C
:102D8000E801D501ED91FC911197EC0FFD1F108129
:102D900010826D917C916E0D7F1DC60161157105CC
:102DA000A1F00E943116F50180819181C80FD91FD1
:102DB0001883C601DF91CF911F910F91FF90EF9083
:102DC000DF90CF90BF90AF9008950E945215EBCF47
:102DD000CF93DF93EC01FB01248135810E949C1687
:102DE000CE01DF91CF9108950F931F93CF93DF937F
:102DF000CDB7DEB72C970FB6F894DEBF0FBECDBFB0
:102E0000FC01248135811216130664F48C012531EE
:102E100031059CF40E94CC0364E170E080E090E016
:102E20000E9482052C960FB6F894DEBF0FBECDBF70
:102E3000DF91CF911F910F9108952FE030E050E086
:102E400040E0BC01CE0107960E949C164B855C8534
:102E50006F8178858AE095E00E949F0369E170E0C8
:102E600080E090E00E9482054FE050E0B801CE0182
:102E700001960E94E816BE016F5F7F4FCE01079654
:102E80000E941915CE0101960E946415CE01079685
:102E90000E94CC0364E170E080E090E00E94820533
:102EA00062E871E0CE0107960E943116CE010796C6
:102EB0000E946415B7CFEF92FF920F931F93CF93A9
:102EC000DF93CDB7DEB7A1970FB6F894DEBF0FBE84
:102ED000CDBF7C01CB01BA01F701118210821382B0
:102EE00012821582148242E0420F8E010F5F1F4F43
:102EF0000E94932F009789F0BC01C7010E943116F0
:102F0000A1960FB6F894DEBF0FBECDBFDF91CF9173
:102F10001F910F91FF90EF900895C7010E945215E5
:102F2000EFCF0F931F93CF93DF93D62FC42F109221
:102F3000840110928301FC01448155814F5F5F4FF2
:102F400021F063E871E00E948114E0919606F0910F
:102F5000970681E896E00995C80F03E811E0F801AB
:102F600021918F01211105C0DF91CF911F910F9108
:102F700008954C2F6D2F81E896E00E945A0CD80FCF
:102F8000EECF8F929F92AF92BF92CF92DF92FF923D
:102F90000F931F93CF93DF93CDB7DEB7AE970FB6E6
:102FA000F894DEBF0FBECDBF6C015B018A010E94A9
:102FB0000E061CA21BA21EA21DA218A61FA228EE6E
:102FC00033E040E050E00E94F636CA01B90120E843
:102FD00031E541E050E00E94F6362AE0AE014F5F55
:102FE0005F4F0E94E72FBE016F5F7F4FCE01839638
:102FF0000E943116BE016D5D7F4FCE0101960E9489
:103000007E166AEE72E0CE0101960E94E715BC01C1
:10301000CE0189960E947E16CE0101960E9464150B
:10302000CE0183960E946415809185069091860654
:103030008D59914071F08DE991E0909386068093CF
:1030400085060E945E038CE593E09093970680933B
:103050009606109298060E945E038FE29CE0909381
:1030600097068093960680918C06803309F0B3C052
:103070008FEF8093A1068093A2068091BA068111FA
:1030800005C081E08093BA060E94030C80908306FD
:1030900090908406E091B206F091B30682E0099523
:1030A000E091B206F091B30681E0099530E020E0AE
:1030B00044E1B40181E896E00E941D0B24EB36E068
:1030C00047E1B40181E896E00E941D0BE091B20651
:1030D000F091B30680E00995BE01675D7F4FCE0198
:1030E00001960E947E1641E060E0CE0101960E94AA
:1030F0009117CE0101960E946415B601CE0101968A
:103100000E947E1641E060E3CE0101960E94911775
:10311000CE0101960E946415B501CE0101960E9470
:103120007E1640E160E0CE0101960E949117CE012B
:1031300001960E946415E0918F06F09190063097F9
:1031400019F081E896E009958090830690908406B6
:10315000E091B206F091B30682E00995E091B206E3
:10316000F091B30681E0099530E020E045E1B4013B
:1031700081E896E00E941D0BF82E882341F024EB95
:1031800036E047E1B40181E896E00E941D0BE09132
:10319000B206F091B30680E00995F1109DCFB80119
:1031A000110F880B990B0E948205CE0189960E940F
:1031B0006415AE960FB6F894DEBF0FBECDBFDF919B
:1031C000CF911F910F91FF90DF90CF90BF90AF9064
:1031D0009F908F900895883231F0823031F081E0F5
:1031E0008093A1064ACF8FEFFBCF83E0F9CFFF9208
:1031F0000F931F93CF93DF93EC01F62E0881198173
:10320000C8010E942635F81621F06F2DC8010E94D2
:103210002E35CE01DF91CF911F910F91FF90089530
:10322000EF92FF920F931F93CF93DF9300D0CDB710
:10323000DEB703EB15E0835B95407C01C701800F8F
:10324000911F9A838983F80161918F01CE010196C4
:103250000E94F718F6E001301F0781F783EB95E035
:103260000F900F90DF91CF911F910F91FF90EF90F2
:103270000895EF92FF920F931F93CF93DF9300D0A7
:10328000CDB7DEB707E016E0875096407C01C70156
:10329000800F911F9A838983F80161918F01CE017C
:1032A00001960E94F718F6E00E321F0781F787E0BB
:1032B00096E00F900F90DF91CF911F910F91FF90AB
:1032C000EF9008952F923F924F925F926F927F926C
:1032D0008F929F92AF92BF92CF92DF92EF92FF9226
:1032E0000F931F93CF93DF93CDB7DEB7E6970FB65B
:1032F000F894DEBF0FBECDBF66E476E082E596E0CF
:103300000E9467160E94A41462E971E0CE01019642
:103310000E948716BE016F5F7F4F82E596E00E9494
:10332000FE14182FCE0101960E946415112329F076
:10333000F0E0E0E0099581E092C066E971E0CE013D
:1033400001960E948716BE016F5F7F4F82E596E06F
:103350000E94FE14182FCE0101960E9464151123BD
:1033600051F16AE971E0CE0101960E9487166EE282
:1033700076E0CE0101960E94FD15BC0188E596E03D
:103380000E946716CE0101960E94641568E576E0FA
:10339000CE0101960E947E16CE0101960E94F4167F
:1033A000CE0101960E94641562E871E088E596E01E
:1033B0000E943116C0CF64EA71E0CE0101960E94EE
:1033C0008716BE016F5F7F4F82E596E00E94FE1474
:1033D000182FCE0101960E946415112359F068EA56
:1033E00071E088E596E00E94311684E396E00E9441
:1033F000C015CCCF66EB71E0CE0101960E94871616
:10340000BE016F5F7F4F82E596E00E94FE14182F89
:10341000CE0101960E9464151123D1F127E030E01E
:1034200046E050E066E476E0CE0101960E949C16EC
:10343000BE016F5F7F4F80E496E00E941915CE01B8
:1034400001960E94641580E496E00E94F314672BB5
:1034500019F41092AE046FCF81E08093AE04E6962B
:103460000FB6F894DEBF0FBECDBFDF91CF911F9195
:103470000F91FF90EF90DF90CF90BF90AF909F9013
:103480008F907F906F905F904F903F902F90089516
:103490006DEB71E0CE0101960E948716BE016F5F51
:1034A0007F4F82E596E00E94FE14182FCE01019610
:1034B0000E946415112309F4B8C08091F303909120
:1034C000F403181619060CF036CF88EC90E09093B0
:1034D0000D0180930C018AE095E00E94A5041BA2D7
:1034E0001CA21DA21EA2CC24C394D12CA0EC2A2E77
:1034F000A3E03A2E5E01F3E2AF0EB11C2E0127E2EB
:10350000420E511CB3EF6B2EB3E07B2E8091F30380
:103510009091F4038C159D050CF40DCF80910C0156
:1035200090910D01813C934024F030920D01209246
:103530000C0100910C0110910D01750148018A18D0
:103540009B08C4018E0D9F1D0E942635F7018193B3
:103550007F01E415F505A9F7C801049690930D01C4
:1035600080930C01EFECEE2EE3E0FE2E0B5C13409B
:10357000C8018E0D9F1D0E942635F70181937F01A2
:103580006E167F06A9F74BA15CA16DA17EA123E079
:10359000CE0145960E945B17BE016B5E7F4FCE0148
:1035A00001960E947E1661EC71E0CE0101960E94A8
:1035B000E715BC0188E596E00E946716CE010196EA
:1035C0000E946415CE0145960E9464156FEC73E06D
:1035D000CE0101960E948716CE0101960E94C01569
:1035E000CE0101960E94641568E576E0CE01019651
:1035F0000E947E16CE0101960E94F416CE0101961D
:103600000E94641580910C0190910D018496909315
:103610000D0180930C0164E170E080E090E00E9475
:103620008205FFEFCF1ADF0A71CF64EC71E0CE01A3
:1036300001960E948716BE016F5F7F4F82E596E07C
:103640000E94FE14182FCE0101960E9464151123CA
:10365000F1F126E030E045E050E066E476E0CE01AE
:1036600001960E949C16BE016F5F7F4F80E496E03A
:103670000E941915CE0101960E94641580E496E01F
:103680000E94F314672B19F41092CE0354CE81E0FC
:103690008093CE0388EC90E090930D0180930C0111
:1036A0001092F4031092F3031092CA031092CB030A
:1036B0001092CC031092CD030E940E066093C603B5
:1036C0007093C7038093C8039093C90334CE6AEC08
:1036D00071E0CE0101960E948716BE016F5F7F4F99
:1036E00082E596E00E94FE14182FCE0101960E94FA
:1036F0006415112309F46DC080914A0690914B0620
:10370000079708F418CE46E050E066E476E0CE0174
:1037100001960E94E816BE016F5F7F4F80E496E03D
:103720000E941915CE0101960E9464150E94292A53
:103730006B017C01C0921701D0921801E09219012F
:10374000F0921A0161ED71E088E596E00E94311671
:1037500022E0B701A601CE0145960E945B17BE018B
:103760006B5E7F4FCE0101960E947E166AEE72E07C
:10377000CE0101960E94E7150E94C015CE01019668
:103780000E946415CE0145960E94641568E576E0B6
:10379000CE0101960E947E16CE0101960E94F4167B
:1037A000CE0101960E9464150E940E0628EE33E0B9
:1037B00040E050E00E94D436CA01B9010E940434AE
:1037C0006093B3047093B4048093B5049093B604EB
:1037D000B2CD6CED71E0CE0101960E948716BE015C
:1037E0006F5F7F4F82E596E00E94FE14182FCE0196
:1037F00001960E946415112309F459C080914A066C
:1038000090914B06079708F496CD46E050E066E4A9
:1038100076E0CE0101960E94E816BE016F5F7F4FF1
:1038200080E496E00E941915CE0101960E9464156D
:103830000E94292A6B017C01C0920801D0920901E3
:10384000E0920A01F0920B0163EE71E088E596E0E8
:103850000E94311621E0B701A601CE0145960E94D3
:103860005B17BE016B5E7F4FCE0101960E947E16F4
:103870006AEE72E0CE0101960E94E7150E94C01523
:10388000CE0101960E946415CE0145960E946415F2
:1038900068E576E0CE0101960E947E16CE01019683
:1038A0000E94F416CE0101960E94641544CD6EEE7E
:1038B00071E0CE0101960E948716BE016F5F7F4FB7
:1038C00082E596E00E94FE14182FCE0101960E9418
:1038D00064151123D9F143E050E066E476E0CE01AF
:1038E00001960E94E816BE016F5F7F4F80E496E06C
:1038F0000E941915CE0101960E94641560E476E0DD
:10390000CE0101960E947E1660E0CE0101960E94D3
:10391000C915BC0184E396E00E946716CE010196AA
:103920000E946415409138065091390641155105A1
:1039300031F065EB75E084E396E00E94811480919C
:103940001501909116010E941019F5CC65EF71E0F8
:10395000CE0101960E948716BE016F5F7F4F82E500
:1039600096E00E94FE14182FCE0101960E94641565
:10397000112309F478C080914A0690914B06409734
:1039800008F027C442E050E066E476E0CE010196FC
:103990000E94E816BE016F5F7F4F80E496E00E94B0
:1039A0001915CE0101960E9464150E94292A20E073
:1039B00030E048EC52E40E9465340E946C3660931B
:1039C000BF057093C0058093C1059093C20562EF57
:1039D00071E088E596E00E9431166091BF05709114
:1039E000C0058091C1059091C2058B019C010059D1
:1039F0001F452140310901341C492105310598F04A
:103A000060E476E0CE0101960E947E1668EF71E0D8
:103A1000CE0101960E94E7150E94C015CE010196C5
:103A20000E94641588CC0E94063420E030E048EC07
:103A300052E40E94FA35AB01BC0122E0CE010196AE
:103A40000E945B17CE0101960E94C015CE0101961F
:103A50000E94641543E050E065E072E088E596E07E
:103A60000E9494156CCF69E072E0CE0101960E942D
:103A70008716BE016F5F7F4F82E596E00E94FE14BD
:103A8000182FCE0101960E9464151123F1F025E054
:103A900030E044E050E066E476E0CE0101960E941A
:103AA0009C16BE016F5F7F4F80E496E00E9419155F
:103AB000CE0101960E94641580E496E00E94F31402
:103AC000709300066093FF053ACF6EE072E0CE017E
:103AD00001960E948716BE016F5F7F4F82E596E0D8
:103AE0000E94FE14182FCE0101960E946415112326
:103AF00009F45EC009E110E0C12CD12C760180E10F
:103B00000E944205BC01990F880B990B0E94063454
:103B10009B01AC01C701B6010E948E356B017C018F
:103B20006AE070E080E090E00E9482050150110997
:103B300031F720E030E040EA50E4C701B6010E94CE
:103B4000653420E030EC4FE754E40E94FA3520E081
:103B500030E048EC51E40E94FA356093DB05709345
:103B6000DC058093DD059093DE0580911501909131
:103B700016010E94101962E172E088E596E00E9449
:103B800031164091DB055091DC056091DD057091A7
:103B9000DE0522E0CE0145960E945B17BE016B5EFA
:103BA0007F4FCE0101960E947E166AE172E062CEDE
:103BB0006DE172E0CE0101960E948716BE016F5F33
:103BC0007F4F82E596E00E94FE14182FCE010196E9
:103BD0000E946415112309F44EC126E030E044E050
:103BE00050E066E476E0CE0101960E949C16BE018C
:103BF0006F5F7F4F80E496E00E941915CE01019619
:103C00000E94641580E496E00E94F3142B017B016E
:103C10006E0185E1C80ED11C6CE572E0C6010E9400
:103C2000871680914A0690914B06298D3A8D5C014A
:103C3000A21AB30A2115310569F1009759F18217CB
:103C4000930740F1A816B90620F05C01E1E0AE1A36
:103C5000B10880904606909047062D893E893EAB7C
:103C60002DABC4010FEF1FEF14012A0C3B1C2816CB
:103C7000390690F06DA97EA90E943239009761F053
:103C80009C0128193909A216B30608F49801019677
:103C90008901EDCF0FEF1FEFA8014F5F5F4F66E483
:103CA00076E0CE0101960E94E816BE016F5F7F4F5D
:103CB00080E496E00E941915CE0101960E946415D9
:103CC000C6010E9464150E94292A4B015C01120161
:103CD00031E0231A31086FE0C6010E940308D8863C
:103CE000CF821D821E82198289E08A8381E08B83C4
:103CF0008C831C8A1B8ACE0101960E94F712CE018A
:103D000001960E940F07CE0101960E94A4130E8116
:103D100010E00530110514F004E010E04BE5441606
:103D2000510408F44DC07FEDC72E75E0D72E812CCD
:103D3000912C5401F12CE12C0E151F05B9F06E2DBC
:103D4000CE0101960E948B129B01AC01F6012193DA
:103D50003193419351936F01C501B4010E948E3597
:103D60004B015C01FFEFEF1AFF0AE6CFB7010F2C02
:103D7000000C880B990B0E9406349B01AC01C50115
:103D8000B4010E94FA354B015C0103EB15E0D12C24
:103D9000C12C0C5F1F4FEC14FD0499F1F80120A514
:103DA00031A542A553A5C501B4010E948D35F80186
:103DB00060A771A782A793A7FFEFCF1ADF0AE9CF09
:103DC0001E141F04CCF50E151F0524F4180121E064
:103DD000221A3108622DCE0101960E948B129B019E
:103DE000AC018101000F111F000F111F01521A4F6A
:103DF000C501B4010E948D35F8016083718382830F
:103E0000938380911501909116010E94101961E22F
:103E100072E088E596E00E94311644E050E066E4E6
:103E200076E0CE0101960E94E816CE0101960E942E
:103E3000C015CE0101962ACDE114F10411F72FED42
:103E4000C22E25E0D22E0E151F05D9F26E2DCE0101
:103E500001960E948B129B01AC01C501B4010E9426
:103E60008D35F60161937193819391936F01FFEF0B
:103E7000EF1AFF0AE8CF67E372E0CE0101960E94D5
:103E80008716BE016F5F7F4F82E596E00E94FE14A9
:103E9000182FCE0101960E946415112309F44BCA14
:103EA00043E050E062E576E0CE0145960E94E816D8
:103EB000BE016B5E7F4FCE0101960E947E1660E0D0
:103EC000CE0101960E94C915BC0180E496E00E94D3
:103ED0006716CE0101960E946415CE0145960E9498
:103EE000641560E476E0CE018F960E947E166BE347
:103EF00072E0CE0101960E9487168BA99CA9892B9E
:103F0000C9F10FA518A969817A81C8010E943239C7
:103F1000009781F19C01201B310B8901CE01019694
:103F20000E94641562E871E0CE0189960E948716AE
:103F300062E871E0CE0183960E9487161016110682
:103F4000E4F46DE372E0CE0101960E948716CE0183
:103F500001960E94F416CE0101960E946415CE01CE
:103F600083960E946415CE0189960E946415CE0145
:103F70008F969ACC0FEF1FEFD1CFBE01615D7F4FBF
:103F8000CE0183960E946716D12CC12C8AEF682E31
:103F900077247A9496E0592E8FA198A5009709F47A
:103FA00009C135E0C316D104C9F36EEF72E0CE014A
:103FB00001960E948716BE016F5F7F4FCE018396E8
:103FC0000E94FE14182FCE0101960E946415111153
:103FD000CAC001E010E0980150E040E0BE016D5D14
:103FE0007F4FCE0145960E949C16BE016B5E7F4FAF
:103FF000CE0101960E947E1660E0CE0101960E94DD
:10400000C915BC01CE0189960E946716CE010196A2
:104010000E946415CE0145960E946415BE01675D3D
:104020007F4FCE0145960E947E16898D9A8D02970C
:1040300008F49CC06EEF72E0CE0101960E948716D4
:10404000BE016F5F7F4FCE0145960E94FE14F82E91
:10405000CE0101960E946415FF2009F487C022E07A
:1040600030E041E050E0BE016B5E7F4FCE01019633
:104070000E949C16CE0101960E94F3144B017B0115
:10408000CE0101960E94641597FE03C04CE1E40E38
:10409000F11CB3016E197F095C9C70015D9CF00CF2
:1040A0001124F701E95FF94F76876587CE014596C0
:1040B0000E946415B701605F794F44E050E0CE0183
:1040C00089960E9481148FEFC81AD80A8FA198A5EB
:1040D0000817190708F067C0A801BE016D5D7F4F82
:1040E000CE0101960E94E816BE016F5F7F4FCE01A0
:1040F00089960E941915CE0101960E946415BE0191
:10410000675D7F4FCE0183960E946716ABA0BCA06F
:10411000A114B10409F440CF0FA118A57501011530
:10412000110509F439CF47019FEF891A990AF70160
:104130008081082E000C990B0E94CE33892BD9F474
:10414000015011090A0D1B1DF8018081082E000C79
:10415000990B0E94CE33892B81F00E151F0568F054
:1041600001501109F1CF02E010E035CFCE014596A4
:104170000E94F31491CF7401D6CF0F5F1F4FA80197
:104180004E195F0958A74FA3AE14BF0420F4B7011E
:10419000C5010E940539EBA1FCA18FA198A5E80FEC
:1041A000F91F1082F9CE62E871E0CE0183960E9479
:1041B0003116F2CEC0920906CC2041F081E0809306
:1041C00007068EE190E00E943919C9CE10920706C9
:1041D000F8CF80E044C92F923F924F925F926F9246
:1041E0007F928F929F92AF92BF92CF92DF92EF9287
:1041F000FF920F931F93CF93DF93CDB7DEB7E49772
:104200000FB6F894DEBF0FBECDBF8C0162E871E03F
:1042100088E596E00E943116C8010596059760F082
:104220008091B704811108C00C3E2FEF120724F0D3
:104230001093B2040093B104F8017A96E432F105C8
:1042400008F0A3C6EA5DFE4D0C9415375227C5272A
:104250004E27C527C527C527C527C527C527C52775
:10426000C5277A217A217A214A21A5237A21A424FB
:104270009B257A217A219E25AD25B025C5277A2157
:104280007A217A217A21BE25272744277A217A218B
:104290007A217A218E010B5E1F4F6FE0C8010E94C8
:1042A000030818870F831D821E82198289E08A8382
:1042B00081E08B838C831C8A1B8ACE0101960E942D
:1042C000F712CE0101960E940F07CE0101960E94BF
:1042D000A413EE80F12C35E0E316F1040CF0F5C0E8
:1042E000E114F10409F0F4C061E076E088E596E0BD
:1042F0000E94671680915C0690915D06892B09F4F7
:10430000C5C068E576E0CE0101960E947E16CE011A
:1043100001960E94F416CE0101960E94641568E58C
:1043200076E0CE0145960E947E168091CE038823CA
:1043300009F4A2C08091F3039091F40384319105B4
:104340000CF09AC000910C0110910D01013CF3E0BA
:104350001F070CF091C001969093F4038093F30330
:104360000E940E06C090C603D090C703E090C80319
:10437000F090C9036C197D098E099F090E940434CD
:1043800020E030E04AE754E40E94FA356093CA0323
:104390007093CB038093CC039093CD03083C11051D
:1043A00034F488EC90E090930D0180930C0180919F
:1043B0000C0190910D010AEC13E09C012A5C334042
:1043C0007901C701800F911F9A838983D8016D916C
:1043D0008D01CE0101960E94F718B3E00E3C1B0739
:1043E00081F7E0900C01F0900D01C70104969093C5
:1043F0000D0180930C01BE016B5E7F4FCE010196D3
:104400000E947E1660E0CE0101960E94C915BC0193
:1044100088E596E00E946716CE0101960E94641519
:1044200040915C0650915D064115510531F06FECED
:1044300073E088E596E00E9481140FEC13E0F70129
:10444000EB5CF3407F01C701800F911F9A83898342
:10445000D8016D918D01CE0101960E94F718B3E04D
:10446000033F1B0781F780910C0190910D01849609
:1044700090930D0180930C01CE0145960E94641526
:1044800062E871E088E596E00E94311664E670E02B
:1044900080E090E00E948205E4960FB6F894DEBFBB
:1044A0000FBECDBFDF91CF911F910F91FF90EF9085
:1044B000DF90CF90BF90AF909F908F907F906F9044
:1044C0005F904F903F902F90089534E0E32EF12CB1
:1044D00062E871E088E596E00E9431162FEDC22E69
:1044E00025E0D22E10E000E0602FCE0101960E9460
:1044F0008B124B015C01D6014D905D906D907D90CB
:104500006D01A3019201C301B2010E94A73681117E
:1045100008C0A3019201C501B4010E948E354B0170
:104520005C010F5F1F4F20E030E04CEF52ECC50103
:10453000B4010E94FF3387FF25C0B801CE018996E0
:104540000E943B166FEB71E0CE0183960E948716A6
:10455000BE01675D7F4FCE0183960E94FD1564EB1F
:1045600071E00E94E71561E076E00E94FD150E946F
:10457000C015CE0183960E946415CE0189960E94D3
:10458000641572C0B3E0EB16F10409F4C2C0B801BF
:10459000CE0189960E943B166FEB71E0CE018396A7
:1045A0000E948716BE01675D7F4FCE0183960E94F1
:1045B000FD15BC018AE396E00E946716CE01839642
:1045C0000E946415CE0189960E94641522E0B5010F
:1045D000A401CE0189960E945B176AE376E0CE01C2
:1045E00083960E947E166CE572E0CE0183960E944F
:1045F000E715BE01675D7F4F0E94FD15BC018AE390
:1046000096E00E946716CE0183960E946415CE0143
:1046100089960E94641568E576E0CE0183960E9433
:104620007E166AE376E0CE0183960E94FD15BC01FA
:1046300088E596E00E946716CE0183960E94641575
:1046400068E576E0CE0183960E947E1660E2CE0198
:1046500083960E94C915BC0188E596E00E94671602
:10466000CE0183960E9464150E151F0509F03CCFFC
:1046700003301105A9F464E572E0CE0183960E942F
:10468000871668E576E0CE0183960E94FD15BC0191
:1046900088E596E00E946716CE0183960E94641515
:1046A0006EE572E080E496E00E94311668E576E0FF
:1046B000CE0189960E947E1660E476E0CE01839654
:1046C0000E947E1644E650E0BE01675D7F4FCE013A
:1046D00083960E94C117CE0183960E946415CE0175
:1046E00089960E94641568E576E0CE0183960E9463
:1046F0007E1666E672E0CE0183960E94E715BC0145
:1047000088E596E00E946716CE0183960E946415A4
:10471000F1CD22E0B501A401CE0183960E945B1782
:10472000BE016D5D7F4FCE0189960E947E1660E2CC
:10473000CE0189960E94C9150E94C015CE018996A6
:104740000E946415CE0183961ACF60E080E10E943A
:1047500011058091B7048111F2C08AE090E0A0E0D9
:10476000B0E089AB9AABABABBCAB69E772E088E574
:1047700096E00E943116312C212C1FA618AAC12CBC
:10478000D12C760102E310E0812C912C540180E1C0
:104790000E944205092E000CAA0BBB0B880E991E25
:1047A000AA1EBB1E65E070E080E090E00E948205DA
:1047B0000150110961F74090DB055090DC056090D5
:1047C000DD057090DE05C501B4010E94063420E0CD
:1047D00030E040EA50E40E94653420E030E040E8F8
:1047E0005AE30E94653420E030E048E452E40E943D
:1047F000FA35A30192010E948D3520E030E040E7B8
:1048000051E40E9465344B015C01A30192016AE905
:1048100079E989E390E40E948D359B01AC01C501E3
:10482000B4010E94FA3520E030E0A9010E948E35E3
:1048300020E030E040E251E40E9465345B018C01ED
:10484000232D322D4FA558A90E94A236181624F404
:104850003A2C2B2C0FA718AB9FEFC91AD90AE90ADB
:10486000F90A89A99AA9ABA9BCA98C159D05AE0521
:10487000BF050CF087CF6EE170E080E090E00E9411
:10488000820560E872E088E596E00E94311622E039
:10489000432D522D6FA578A9CE0101960E945B177A
:1048A000BE016F5F7F4FCE0145960E947E166DE878
:1048B00072E0CE0145960E94E715BC0180E496E0C7
:1048C0000E946716CE0145960E946415CE0101969E
:1048D0000E94641568E576E0CE0145960E947E163A
:1048E00060E476E0CE0101960E947E1644E650E038
:1048F000BE016B5E7F4FCE0101960E94C117CE01B3
:1049000001960E946415CE0145960E94641564E9E3
:1049100072E0CE0101960E94871660E476E0CE0137
:1049200001960E94FD1568E576E00E94FD15BC0128
:1049300088E596E00E946716CE010196E7CE83E0F7
:1049400090E0A0E0B0E00DCF68EC70E080E090E097
:104950000E9482050E940E1064E670E080E090E004
:104960000E94820562E370E080E090E00E94820590
:1049700049E050E067E271E08EE596E00E949F0317
:1049800062E370E080E090E00E94820503E010E0C6
:104990008EE596E00E94A408892B61F149E050E081
:1049A00067E271E08EE596E00E949F0365E070E0AB
:1049B00080E090E00E948205F12CE12C8EE596E0EB
:1049C0000E94A40892E0E916F104A4F48EE596E0B2
:1049D0000E94A408892B39F08EE596E00E94BC085D
:1049E000AFEFEA1AFA0A65E070E080E090E00E941A
:1049F0008205E4CF62E370E080E090E00E948205EF
:104A00000150110929F68AE090E00E94A7106B017D
:104A10007C0120E030E0A9010E94FF33181634F039
:104A20008AE090E00E94A7106B017C010BE010E08F
:104A300020E030E042ED53E4C701B6010E94FF33AD
:104A4000181684F00150110969F068EC70E080E0FC
:104A500090E00E94820583E090E00E94A7106B0125
:104A60007C01E6CF20E030E0A901C701B6010E9439
:104A7000FF3318160CF038CC20E030E048EC52E45C
:104A8000C701B6010E94FF3321E087FF20E0B70194
:104A9000A601CE0101960E945B17BE016F5F7F4F9A
:104AA00088E596E00E941915CE0101960E946415D2
:104AB00068E576E0CE0101960E947E1668E972E014
:104AC000CE0101960E94E715BC0188E596E00E94A0
:104AD0006716CE0101960E9464156CE972E080E4CD
:104AE00096E00E94311668E576E0CE0101960E94BC
:104AF0007E1660E476E0CE0145960E947E1644E67E
:104B000050E0BE016F5F7F4FCE0145960E94C117F6
:104B1000CE0145960E946415CE0101960E9464154F
:104B200066EA72E0CE0101960E94871668E576E09B
:104B3000CE010196FACE0E940E06DCCB8091B7041E
:104B4000882321F088E596E00E94CC0368EC70E0B1
:104B500080E090E00E948205CDCB1092B704CACBD2
:104B600081E08093B70480930F068091B104909107
:104B7000B2049093B0048093AF04BCCB8BE0C82EFA
:104B8000D12CF12CE12C11E066246A9405EE95EC11
:104B9000792E1093E604B3E2B09308051092E7046F
:104BA000109209050E945D051B012C018091E00413
:104BB000811161C01093E0041093DF046092DE0461
:104BC0001092DD041093DC041093BB048091BB04AD
:104BD00086648093BB048091BA04813009F010C1CF
:104BE0001092BA040E945D051B012C018091BB0448
:104BF0008093BB008091E2049091E304A091E404CF
:104C0000B091E504892B8A2B8B2BA1F00E945D05C6
:104C10002091E2043091E3044091E4045091E504D2
:104C20006219730984099509261737074807590738
:104C300008F442C08091BC0083FDD8CF7092BC00C4
:104C40000E945D051B012C018091E004813009F474
:104C5000DAC08091DD04823008F0F7C08091DD0475
:104C6000ECEBF4E0A5EFB3E090E0981751F121915F
:104C70002D939F5FFACF8091E2049091E304A0917D
:104C8000E404B091E504892B8A2B8B2B09F48ECF99
:104C90000E945D052091E2043091E3044091E40418
:104CA0005091E5046219730984099509261737079D
:104CB0004807590708F07ACF8091E1040E9438092B
:104CC00080E01092AB048093AA0487EA95E00E94EA
:104CD000580A982E812C87EA95E00E94580A5C01B8
:104CE000A828B92881E00E945909B50190E080E028
:104CF0000E9404342AE939E949E95FE30E94FA3560
:104D00000E947336E616F70608F47B0162E370E052
:104D100080E090E00E948205E1E0CE1AD10809F01F
:104D200038CF6BEA72E088E596E00E9431161E8A61
:104D30001D8A188E1F8A1A8E198E4AE0BE016F5F77
:104D40007F4FC7010E942D30BE016F5F7F4FCE01A4
:104D500045960E943116BE016B5E7F4FCE010196D3
:104D60000E947E166BEB72E0CE0101960E94E71561
:104D7000BC0180E496E00E946716CE0101960E9475
:104D80006415CE0145960E94641568E576E0CE0173
:104D900001960E947E1660E476E0CE0145960E9460
:104DA0007E1644E650E0BE016F5F7F4FCE01459610
:104DB0000E94C117CE0145960E946415CE0101964E
:104DC0000E94641560EC72E0CE0101960E94871685
:104DD00060E476E0CE0101960E94FD1568E576E07C
:104DE0000E94FD15BC0188E596E00E946716CE0181
:104DF00001960E94641562E370E080E090E0AACE24
:104E00000093BC001DCF8091E2049091E304A09137
:104E1000E404B091E504892B8A2B8B2B09F414CF81
:104E20000E945D052091E2043091E3044091E40486
:104E30005091E5046219730984099509261737070B
:104E40004807590708F000CF37CF82E009CF81E04B
:104E500080930E010E94B5058C0163EC72E088E539
:104E600096E00E94311660E074E0601B710BCE0189
:104E700001960E943B16CE0101960E94C015CE01FC
:104E800001960E94641536CA63ED72E088E596E0EB
:104E90000E9431160E94B505BC01E9CFF0E0E0E0C8
:104EA000099528CA8091090618160CF055C081E0B2
:104EB000809307066EED72E088E596E00E94311659
:104EC00080910706882309F44AC06CEE72E0CE0197
:104ED00001960E94871668E576E0CE0101960E9451
:104EE000FD15BC0188E596E00E946716CE0101968B
:104EF0000E94641568E576E0CE0101960E947E1658
:104F0000CE0101960E94F416CE0101960E9464150E
:104F100068EE73E080E090E00E94820580910706D1
:104F200081110E94CC2762E871E088E596E00E943A
:104F300031168091B70480930F068111DBC96DEFA4
:104F400072E08CE496E00E94311686EE9FEF90931B
:104F5000B2048093B104CEC910920706ABCF64EFC0
:104F600072E0CE0101960E94871668E576E0CE01D8
:104F700001960E94FD15BC0188E596E00E94671627
:104F8000CE0101960E946415D4CF60E073E088E5FD
:104F900096E00E943116AEC90F931F93CF93DF9313
:104FA00007E016E0D0E0C0E00A5F1F4F80910906DD
:104FB000082E000C990BC817D9076CF4F8018781EB
:104FC00090850E94EB2068EE73E080E090E00E9404
:104FD00082052196E9CFDF91CF911F910F9108951E
:104FE0001F920F920FB60F9211242F933F934F935E
:104FF0005F936F937F938F939F93AF93BF93EF9341
:10500000FF938AE095E00E943604FF91EF91BF91F3
:10501000AF919F918F917F916F915F914F913F9150
:105020002F910F900FBE0F901F9018951F920F9207
:105030000FB60F9211242F938F939F93EF93FF93AB
:10504000E0911A05F0911B058081E0912005F09117
:10505000210582FD1BC09081809123058F5F8F7396
:1050600020912405821741F0E0912305F0E0E65FEE
:10507000FA4F958F80932305FF91EF919F918F9128
:105080002F910F900FBE0F901F9018958081F4CF35
:105090001F920F920FB60F9211242F933F938F936D
:1050A0009F93AF93BF9380919E0490919F04A09192
:1050B000A004B091A10430919D0423E0230F2D376B
:1050C00058F50196A11DB11D20939D0480939E0467
:1050D00090939F04A093A004B093A1048091A20494
:1050E0009091A304A091A404B091A5040196A11DE0
:1050F000B11D8093A2049093A304A093A404B09341
:10510000A504BF91AF919F918F913F912F910F90E7
:105110000FBE0F901F90189526E8230F0296A11D31
:10512000B11DD2CF1F920F920FB60F9211242F9361
:105130003F934F935F936F937F938F939F93AF931F
:10514000BF93EF93FF93E0919B04F0919C04309701
:1051500049F0A685B7858585968D91FF14C09C91F1
:105160008923A1F4FF91EF91BF91AF919F918F910E
:105170007F916F915F914F913F912F910F900FBE53
:105180000F901F9018959C91892361F7A389B4898A
:105190009C918589809589238C938689978901972D
:1051A000F1F7608D718DA685B785558538E020E0D3
:1051B000CB010197F1F7822F90E095958795282FE5
:1051C0004C91452309F02068315091F7868D81FD7F
:1051D00020958091990490E001968F7399273091E2
:1051E0009A04381799F0A0919904B0E0A75ABB4FE0
:1051F0002C9380939904828D938D0197F1F7A38965
:10520000B4898C919589892B8C93ACCF868D8160E4
:10521000868FF1CF1F920F920FB60F9211242F930A
:105220003F934F935F936F937F938F939F93AF932E
:10523000BF93EF93FF938091B900887F803609F484
:105240004AC0F0F5883209F4A7C018F5803109F496
:105250009BC0B8F4882309F4F9C0883009F494C0DD
:10526000FF91EF91BF91AF919F918F917F916F913E
:105270005F914F913F912F910F900FBE0F901F9014
:105280001895883109F488C0803251F78093DE0484
:1052900014C0803409F49DC040F48033B9F38833DE
:1052A000F9F68093DE0485ECB0C0803509F485C042
:1052B000883509F496C0883499F60E94BB14D0CF83
:1052C000883909F48CC038F5883729F050F48836CD
:1052D00011F0803729F683E08093E004109258049F
:1052E00057C0883809F47BC0803919F0803809F03C
:1052F000B7CF80915804803208F071C0E091580413
:1053000081E08E0F809358048091BB00F0E0E85C50
:10531000FB4F80833DC0803B39F0E0F4803A09F4D4
:1053200079C0883A09F09CCF84E08093E004109221
:10533000370410923604E091A804F091A90409956D
:105340008091360481110FC081E080933604109261
:10535000160409C0803C09F4A6CF883C09F4A3CF09
:10536000883B09F07DCFE091370481E08E0F809378
:105370003704F0E0EA5EFB4F80818093BB009091A0
:1053800037048091360429C08091BB048093BB0010
:1053900085EC8093BC0064CF9091DD048091DC04A7
:1053A000981758F5E091DD0481E08E0F8093DD04BD
:1053B000F0E0E454FB4F8081E9CFE091DD0481E02F
:1053C0008E0F8093DD048091BB00F0E0E454FB4F2E
:1053D00080839091DD048091DC049817C8F285E801
:1053E000D8CFE091DD0481E08E0F8093DD048091C1
:1053F000BB00F0E0E454FB4F80838091DF04811117
:105400005CCF81E08093BA0484EA8093BC00109260
:10541000E00426CF85EC8093BC001092E0048091DC
:105420005804803230F4E0915804F0E0E85CFB4F1F
:1054300010826091580470E0E091A604F091A704F6
:1054400088E394E00995109258040ACF1092DE0484
:1054500034CF8091400690914106009711F00C9452
:10546000B12F60E070E0CB010895CF9310920D054D
:1054700010920C0588EE93E0A0E0B0E080930E055A
:1054800090930F05A0931005B093110522E431E02D
:1054900030930B0520930A0525EC30E03093170577
:1054A0002093160524EC30E030931905209318055D
:1054B00020EC30E030931B0520931A0521EC30E0FE
:1054C00030931D0520931C0522EC30E030931F051E
:1054D00020931E0526EC30E0309321052093200513
:1054E000109223051092240510922505109226058E
:1054F0001092AA051092A9058093AB059093AC0574
:10550000A093AD05B093AE0584E591E09093A80516
:105510008093A7051092800610927F0688E791E09D
:1055200090937E0680937D061092B8061092B9067D
:105530001092BA061092860610928506109288067E
:105540001092870610928A0681E08093890682E293
:1055500080938B061092900610928F06E4EAF6E094
:1055600082EB96E02FEF21938E179F07E1F7C1E0C2
:10557000C093A1068CE593E09093970680939606DE
:10558000C09398061092990610929A0680E4809330
:105590009B0610929C068BE593E09093B306809354
:1055A000B2068BE191E0909384068093830610927B
:1055B000AF060E94030C88E791E090937E068093EB
:1055C0007D06109261061092600688EE93E0A0E0DE
:1055D000B0E08093620690936306A0936406B09354
:1055E000650686E691E090935F0680935E061092D2
:1055F0007506109274061092770610927606109235
:1056000079061092780610927B0610927A068091A5
:105610007C068E7F8D7F80937C0681FB662760F9F8
:105620006C2789E00E94C50461E089E00E941105B1
:10563000E2E5F6E0E491E0936E06EEE3F6E0E49155
:10564000F0E0EE0FFF1FE55DF94F85919491909387
:10565000700680936F0660E08AE00E9411058091D9
:105660007C0681FD04C061E08AE00E94C5048AE0F6
:1056700080936A06E3E5F6E0E491E0936B06EFE3DE
:10568000F6E0E491F0E0EE0FFF1FEF5DF94F85913A
:10569000949190936D0680936C0662E871E088E5C2
:1056A00096E00E94871662E871E082E596E00E942B
:1056B000871662E871E08CE496E00E94871662E843
:1056C00071E086E496E00E94871662E871E080E46B
:1056D00096E00E94871662E871E08AE396E00E94F5
:1056E00087166EE073E084E396E00E94871665E11A
:1056F00073E08EE296E00E9487161092070685E01E
:10570000809308061092090610920B0610920A0662
:1057100010920D0610920C0610920E0610920F06B3
:105720006FE173E081E096E00E94871686E190E0E9
:105730009093B4058093B3058CE79CE8A1E0B0E0BA
:105740008093BF059093C005A093C105B093C20597
:1057500081EA97E6A3E3BDEB8093C3059093C4056C
:10576000A093C505B093C60586E696E6A6EABFE314
:105770008093C7059093C805A093C905B093CA0547
:105780001092CB051092CC051092CD051092CE054B
:105790001092CF051092D0051092D1051092D2052B
:1057A00081E08093D30529E130E03093D505209343
:1057B000D4058093D60580E090E4ACE1B5E4809315
:1057C000D7059093D805A093D905B093DA05109228
:1057D000DB051092DC051092DD051092DE05EFED81
:1057E000F5E080E1DF011D928A95E9F71092EF055F
:1057F0001092F0051092F1051092F2051092F30547
:105800001092F4051092F5051092F6051092F70526
:105810001092F8051092F9051092FA051092FB0506
:105820001092FC051092FD051092FE0581E090E0BB
:10583000909300068093FF05CF910895CF93DF9357
:10584000CDB7DEB72C970FB6F894DEBF0FBECDBF35
:10585000789484B5826084BD84B5816084BD85B54B
:10586000826085BD85B5816085BD80916E00816057
:1058700080936E00109281008091810082608093FD
:1058800081008091810081608093810080918000FF
:105890008160809380008091B10084608093B1002A
:1058A0008091B00081608093B00080917A00846024
:1058B00080937A0080917A00826080937A00809150
:1058C0007A00816080937A0080917A00806880936A
:1058D0007A001092C10061E08EE00E941105E09113
:1058E0001A05F0911B0582E08083E0911605F09186
:1058F00017051082E0911805F09119058FEC80834F
:1059000010922205E0911E05F0911F0586E080832C
:10591000E0911C05F0911D05808180618083E091FC
:105920001C05F0911D05808188608083E0911C0535
:10593000F0911D05808180688083E0911C05F091C5
:105940001D0580818F7D808360E08EE00E94C5040C
:105950001092AB041092AA041092E7041092090569
:105960000E941A098CE993E09093A9048093A804FB
:105970008DE993E09093A7048093A60481E080933F
:10598000E60483E28093080560E187EA95E00E94DF
:105990009F0A81E00E9459098FE39CE90197F1F782
:1059A00000C0000068EC70E080E090E00E9482059A
:1059B00084E690E090931601809315010E942635AD
:1059C0008093AC0485E690E00E9426358093AD0478
:1059D0000091AC041091AD04B801012E000C880BAD
:1059E000990B0E9406349B01AC010E94A7368111DD
:1059F00006C00B5011090C30110508F407C184E6EC
:105A000090E00E94101937E0E32E36E0F32E670194
:105A10000EE110E0C8010E942635F60181936F0166
:105A20000F5F1F4F07321105A9F710910806612F6C
:105A3000012E000C770B880B990B0E9406349B01FA
:105A4000AC010E94A736811103C0153009F401C1D1
:105A50008EE190E00E94391968EC70E080E090E0FF
:105A60000E9482056BE273E088E596E00E943116A1
:105A70001092AB041092AA041092E7041092090548
:105A80000E941A098CE993E09093A9048093A804DA
:105A90008DE993E09093A7048093A60464E670E0F8
:105AA00080E090E00E94820563E871E0CE010196FB
:105AB0000E948716CE0101960E94F416CE0101962F
:105AC0000E9464158091830690918406F1E08F30E6
:105AD0009F0751F090931201809311018FE091E0A4
:105AE000909384068093830681E49BE09093100159
:105AF00080930F0181E896E00E94E10B68E576E073
:105B0000CE0101960E947E1664E376E0CE010796F0
:105B10000E947E1648EE53E0BE016F5F7F4FCE01BC
:105B200007960E94C117CE0107960E946415CE0108
:105B300001960E94641564E376E0CE0101960E940E
:105B40007E1660E0CE0101960E94C9150E94C01524
:105B5000CE0101960E94641568E576E0CE010196BB
:105B60000E947E16CE0101960E94F416CE01019687
:105B70000E9464158AE2C82ED12C98EE892E93E0FB
:105B8000992EA12CB12C20E0E22E20E0F22E01E093
:105B900062E871E086E496E00E94311662E871E006
:105BA000CE0107960E94871610E08AE095E00E94D9
:105BB0001604181619060CF05AC0111158C08AE0C4
:105BC00095E00E94F4038A3009F001C11091AE04FF
:105BD000112309F411C180914A0690914B06892B3B
:105BE00009F403C164E373E0CE0101960E948716B5
:105BF000BE01695F7F4FCE0101960E94FD150E9494
:105C0000CC03CE0101960E946415EFC043EBE42E55
:105C100045E0F42E04E610E0C8010E942635F701A5
:105C200081937F010F5F1F4F023B1105A9F765EBC1
:105C300075E0CE0101960E948716BE016F5F7F4F0F
:105C400084E396E00E941915CE0101960E94641526
:105C5000DACE0EE110E0C8010E942635F7018193EB
:105C60007F010F5F1F4F05341105A9F7F5CE8B8516
:105C70009C85892B51F08AE095E00E94A50464E19F
:105C800070E080E090E00E948205BE01695F7F4F76
:105C900086E496E00E941915CE0107960E946415CD
:105CA00062E871E088E596E00E94311680914A062C
:105CB00090914B068130910509F0C6C066E476E00C
:105CC00082E596E00E9467160E94A41462E576E0E1
:105CD000CE0101960E947E168D819E81892B09F44A
:105CE000A5C0E981FA81309709F4A0C0808182348F
:105CF00009F484C0833409F48EC0813409F096C05D
:105D00006DE373E086E496E00E943116CE010196C1
:105D10000E94641586E496E00E94F314CB010E9471
:105D2000EB208091B704882309F43FC00E940E063F
:105D3000A50194010E94D436CA01B9010E9404341D
:105D40002091B3043091B4044091B5045091B6044D
:105D50000E948D3520911701309118014091190151
:105D600050911A010E94A2361816FCF48091B104D9
:105D70009091B2044A9609F4A0C08091AF0490912A
:105D8000B0040E94EB200E940E06A50194010E941F
:105D9000D436CA01B9010E9404346093B3047093ED
:105DA000B4048093B5049093B6046AE070E080E098
:105DB00090E00E948205E114F10409F4E9CE0E940A
:105DC0002204882309F4E4CE0E940000E1CE8D3045
:105DD00009F4FCCE89831A8241E050E0BE016F5F76
:105DE0007F4FCE0107960E9494156AE070E080E034
:105DF00090E00E948205D9CE11E0F7CF60E473E015
:105E000086E496E00E9431161092B7048CEF9FEF63
:105E10000E94EB207BCF63E473E086E496E00E946F
:105E200031160093B7048DEF9FEFF2CFBE016F5F85
:105E30007F4F86E496E00E9467166AE070E080E09B
:105E400090E00E94820562CF049768F56EEF72E0E1
:105E5000CE0101960E948716BE016F5F7F4F86E4D8
:105E600096E00E94FE14182FCE0101960E94641540
:105E70001123C9F080914A0690914B06029788F051
:105E8000E0914606F0914706309759F081818033C2
:105E90000CF4845E9601281B310987FD3395C901F6
:105EA0003ECF80E0F6CF80914A0690914B06029754
:105EB00008F437CF0E94621934CF809107068823F7
:105EC00009F461CF0E94CC275ECF81E096E00E946A
:105ED00064158EE296E00E94641584E396E00E94C9
:105EE00064158AE396E00E94641580E496E00E94BF
:105EF000641586E496E00E9464158CE496E00E94A6
:105F0000641582E596E00E94641588E596E00E949B
:105F1000641586E691E090935F0680935E068EE5B9
:105F200096E00C94DD08EF920F931F93CF93DF93CD
:105F3000E80134E047FD34E1042E000C550B57FF17
:105F400003C0519541955109E32E022F242FAE0134
:105F50000E944730CE01DF91CF911F910F91EF90BA
:105F60000895662777270C94A6311F93FC01992783
:105F70008827BC01E89411911032E9F3193010F030
:105F80001E30C8F31B3251F01D3249F4689406C02C
:105F90000E94F62F610F711D811D911D11911053EB
:105FA0001A30B0F33EF490958095709561957F4FCF
:105FB0008F4F9F4F1F910895BB274A3031F499238B
:105FC00022F4BDE2909581959F4F0C942E30BB2713
:105FD0002A3051F4992342F4BDE290958095709552
:105FE00061957F4F8F4F9F4F0C940C30592F482F46
:105FF000372F262F660F771F881F991F660F771F71
:10600000881F991F620F731F841F951F660F771FCC
:10601000881F991F0895BB27FA01A62F62177105E3
:1060200081059105330B30FB66F0AA27660F771FB9
:10603000881F991FAA1FA21710F0A21B6395385042
:10604000A9F7A05DAA3308F0A95DA19336F7B111B5
:10605000B1931082CA010C94EF33BB27FB01552783
:10606000AA27880F991FAA1FA41710F0A41B8395B5
:106070005051B9F7A05DAA3308F0A95DA19300972C
:1060800079F7B111B1931192CB010C94EF33A9E0E0
:10609000B0E0EDE4F0E30C944D356A01F22EB02E41
:1060A000102FFBE3AF2EA01608F41BE31F5F012F98
:1060B00027E0AE014F5F5F4F0E94F632BC0189813D
:1060C000982F9970913009F43FC09BE2E1FC04C025
:1060D0009E2D9170E0FC3AC05E2D5071E82FE87063
:1060E00083FF46C084E0911101C083E0EF2DE81BDF
:1060F0008F1508F0E0E0D6018E2F20E2552351F1F4
:10610000992329F0D6019C93C60101966C01960152
:106110002D5F3F4FE2FE24C08EE4D6018C9391E4C4
:1061200011969C93119712968C93D9018E2F90E221
:1061300081111BC0E20FF32FF11D10828EEF9FEF34
:106140002996ECE00C9469359DE2C6CF90E2C4CF6D
:106150002D9381508111FCCFCE0ED11CE0E0D0CF29
:106160008EE6D6018C9391E6DBCF9D938150E0CFF4
:10617000482F447082FF3DC084E0911101C083E04C
:106180008F1510F4EF2DE81BD6018E2F20E255233A
:1061900009F1992329F0D6019C93C60101966C015F
:1061A00096012D5F3F4FE2FE1BC089E4D6018C9320
:1061B0008EE411968C93119786E412968C93D901F4
:1061C0008E2F90E2882309F4B5CF9D938150FACFAA
:1061D0002D9381508111FCCFCE0ED11CE0E0D9CFA0
:1061E00089E6D6018C938EE611968C93119786E6FC
:1061F000E4CF9B0177FF02C030E020E0A1E0B0E0F7
:10620000911102C0B0E0A0E0F9013196AE0FBF1FBE
:106210008B2C912CBB2009F461C05401EFEFAE1A16
:10622000BE0AAA0DBB1DFA161B0619F014F04F2D5D
:106230004A1B511188C0E3FC59C07601A42FB0E27B
:10624000A1114FC0C40ED11C992309F45BC040E0DA
:10625000D6011196F60190836D01552309F448C0CB
:10626000012F060F9A81582F507184FF03C091337C
:1062700009F4015010160CF047C0093008F008E08E
:10628000EEE2FE2E5B01A01AB10885019194819483
:1062900091082F3F320729F4D601FC92F60131967E
:1062A0006F016217730794F1021713077CF5DB0186
:1062B000A21BB30BAA24A394B12CAC0EBD1EAA0D35
:1062C000BB1D11968C9121503109D60111962815CC
:1062D0003905F4F0F60180836D01DBCFB12CA12CE0
:1062E000A0CFF701B1937F01A150AACF9111B0CFF8
:1062F000D601942F50E302C05D9391509111FCCFD1
:10630000C40ED11C40E0ACCF01E0BACF80E3DBCFBC
:106310006217730731F4963388F4953311F45523DB
:1063200069F0F6018083FD01842F90E2811108C09D
:10633000A40FB11D1C9290E080E002CF81E3F1CF69
:1063400091938150F3CF911183CF8ACFB0E0A0E039
:10635000ECEAF1E30C944D355C017B0161157105AC
:1063600019F0DB018D939C9385010F5F1F4FF501A1
:10637000D0818D2F90E00E94CE336C01892BB9F52E
:10638000DD32B9F50F5F1F4FD5011196DC91C1E0E9
:106390005801F1E0AF1AB10843E050E060E770E067
:1063A000C5010E94D733892B69F5680182E0C80EC8
:1063B000D11C45E050E06BE670E0C6010E94D73387
:1063C000892B21F4680197E0C90ED11CE114F10476
:1063D00019F0D701CD92DC9260E070E080E89FEF89
:1063E000C111FFC060E070E080E89FE7FAC058018B
:1063F000BBCFDB3229F485010E5F1F4FF501D18140
:10640000C0E0C6CF43E050E068E670E0C5010E94FE
:10641000D733892BE9F0F80110E000E020E030E00C
:10642000A9015F01B0ED8B2E8D0E89E08815C8F1B2
:106430009C2E689491F88C2F8870C2FF16C0811131
:1064400002C00F5F1F4F3196D501DC91C92DE9CFF6
:10645000E114F10429F00E5F1F4FF701118300834F
:1064600060E070E080EC9FE7BCC0882311F0015031
:106470001109A5E0B0E00E943C359B01AC01220F60
:10648000331F441F551F280D311D411D511D283933
:1064900099E93907490799E15907A8F2C6609C2E86
:1064A000D2CFAEEF8A1206C0C3FD3CC09C2E6894CA
:1064B00093F8C9CFDF7DD534A9F580818D3239F4C9
:1064C000C061DF011296818162E070E006C0DF01E9
:1064D0008B32C1F3119661E070E080535D01A61A22
:1064E000B70A8A30F8F4E0E8CE16ECE0DE065CF499
:1064F000B601660F771F660F771FC60ED71ECC0C2E
:10650000DD1CC80ED11C5D01FFEFAF1ABF0A8C91D4
:1065100080538A30A8F1C4FF03C0D194C194D1083C
:106520000C0D1D1DC1FF09C0E114F10431F081E023
:10653000A81AB108D701AD92BC92CA01B9010E9454
:106540000434C370C33009F490584B015C0120E05F
:1065500030E0A9010E94FF33882309F440C0CFE94D
:10656000D0E017FF05C0119501951109C7E8D0E0EB
:106570006E01B8E1CB1AD10880E2E82EF12C0FC0F1
:10658000D501B1CFFE0125913591459154910E1958
:106590001F09C501B4010E9465344B015C01D5019E
:1065A000C4010E151F0574F72497F594E794CC16D3
:1065B000DD06A9F78A2F880F8B2F881F8F3F49F0A0
:1065C00020E030E0A901C501B4010E94FF33811130
:1065D00006C082E290E09093BC068093BB06C501A2
:1065E000B401CDB7DEB7ECE00C946935283008F083
:1065F00027E03327DA01990F311D87FD916000965E
:106600006105710539F432602E5F3D9330E32A95C0
:10661000E1F708959F3F30F080387105610509F07A
:106620003C5F3C5F3D93913008F08068911DDF93A3
:10663000CF931F930F93FF92EF92192F987F969508
:10664000E92F96959695E90FFF27E350FF4F99277D
:106650003327EE24FF24A701E7010590089407944F
:1066600028F4360FE71EF81E491F511D660F771FCD
:10667000881F991F0694A1F70590079428F4E70E48
:10668000F81E491F561FC11D770F881F991F661FCF
:106690000694A1F70590079428F4F80E491F561F99
:1066A000C71FD11D880F991F661F771F0694A1F77A
:1066B0000590079420F4490F561FC71FD81F990F44
:1066C000661F771F881F0694A9F78491109517708D
:1066D00041F0D695C79557954795F794E7941A9545
:1066E000C1F7E3EAF0E06894159015913591659152
:1066F000959105907FE27395E118F10A430B560BD3
:10670000C90BD009C0F7E10CF11E431F561FC91F6A
:10671000D01D7EF4703311F48A95E6CFE8940150D1
:1067200030F0080F0AF40027021708F4202F2395F1
:10673000022F7A3328F079E37D932A95E9F710C088
:106740007D932A9589F606949795679537951795C1
:106750001794E118F10A430B560BC90BD00998F0B6
:1067600023957E9173957A3308F070E37C93201320
:10677000B8F77E9170617D9330F0839571E37D93DE
:1067800070E32A95E1F71124EF90FF900F911F918C
:10679000CF91DF91992787FD9095089591110C94E1
:1067A000D234803219F089508550C8F70895FB0122
:1067B000DC014150504088F08D9181341CF08B35C4
:1067C0000CF4805E659161341CF06B350CF4605EF6
:1067D000861B611171F3990B0895881BFCCFDC01B6
:1067E000FC01672F71917723E1F7329704C07C9108
:1067F0006D9370836291AE17BF07C8F308950E942E
:10680000413408F481E00895E89409C097FB3EF410
:1068100090958095709561957F4F8F4F9F4F9923ED
:10682000A9F0F92F96E9BB279395F695879577956B
:106830006795B795F111F8CFFAF4BB0F11F460FF2B
:106840001BC06F5F7F4F8F4F9F4F16C0882311F083
:1068500096E911C0772321F09EE8872F762F05C097
:10686000662371F096E8862F70E060E02AF09A9532
:10687000660F771F881FDAF7880F9695879597F927
:106880000895990F0008550FAA0BE0E8FEEF1616C1
:106890001706E807F907C0F012161306E407F50714
:1068A00098F0621B730B840B950B39F40A2661F088
:1068B000232B242B252B21F408950A2609F4A1402B
:1068C000A6958FEF811D811D08950E9478340C9448
:1068D000EC340E94DE3438F00E94E53420F0952339
:1068E00011F00C94D5340C94DB3411240C94203525
:1068F0000E94FD3470F3959FC1F3950F50E0551F32
:10690000629FF001729FBB27F00DB11D639FAA2704
:10691000F00DB11DAA1F649F6627B00DA11D661F53
:10692000829F2227B00DA11D621F739FB00DA11D74
:10693000621F839FA00D611D221F749F3327A00D2E
:10694000611D231F849F600D211D822F762F6A2FCA
:1069500011249F5750409AF0F1F088234AF0EE0F2F
:10696000FF1FBB1F661F771F881F91505040A9F75C
:106970009E3F510580F00C94D5340C9420355F3F38
:10698000E4F3983ED4F3869577956795B795F79598
:10699000E7959F5FC1F7FE2B880F911D9695879510
:1069A00097F9089599278827089597F99F6780E8B0
:1069B00070E060E008959FEF80EC089500240A9451
:1069C0001616170618060906089500240A941216CA
:1069D0001306140605060895092E0394000C11F4FD
:1069E000882352F0BB0F40F4BF2B11F460FF04C0AA
:1069F0006F5F7F4F8F4F9F4F089557FD9058440F03
:106A0000551F59F05F3F71F04795880F97FB991F0D
:106A100061F09F3F79F087950895121613061406CA
:106A2000551FF2CF4695F1DF08C016161706180657
:106A3000991FF1CF86957105610508940895E89432
:106A4000BB2766277727CB0197F90895F999FECFE1
:106A500092BD81BDF89A992780B50895262FF9999E
:106A6000FECF1FBA92BD81BD20BD0FB6F894FA9A31
:106A7000F99A0FBE019608950E947E35A59F900D4C
:106A8000B49F900DA49F800D911D112408952F9205
:106A90003F924F925F926F927F928F929F92AF92AE
:106AA000BF92CF92DF92EF92FF920F931F93CF93FB
:106AB000DF93CDB7DEB7CA1BDB0B0FB6F894DEBF92
:106AC0000FBECDBF09942A88398848885F846E84B8
:106AD0007D848C849B84AA84B984C884DF80EE8002
:106AE000FD800C811B81AA81B981CE0FD11D0FB60B
:106AF000F894DEBF0FBECDBFED010895A29FB00197
:106B0000B39FC001A39F700D811D1124911DB29FE1
:106B1000700D811D1124911D08955058BB27AA277F
:106B20000E94A5350C94EC340E94DE3438F00E94AB
:106B3000E53420F039F49F3F19F426F40C94DB344B
:106B40000EF4E095E7FB0C94D534E92F0E94FD3458
:106B500058F3BA17620773078407950720F079F492
:106B6000A6F50C941F350EF4E0950B2EBA2FA02D30
:106B70000B01B90190010C01CA01A0011124FF27EA
:106B8000591B99F0593F50F4503E68F11A16F040E5
:106B9000A22F232F342F4427585FF3CF46953795E4
:106BA0002795A795F0405395C9F77EF41F16BA0BA9
:106BB000620B730B840BBAF09150A1F0FF0FBB1F57
:106BC000661F771F881FC2F70EC0BA0F621F731FA0
:106BD000841F48F4879577956795B795F7959E3FFD
:106BE00008F0B0CF9395880F08F09927EE0F97958E
:106BF000879508950E940E360C94EC340E94E5347B
:106C000058F00E94DE3440F029F45F3F29F00C94E4
:106C1000D53451110C9420350C94DB340E94FD3492
:106C200068F39923B1F3552391F3951B550BBB27BB
:106C3000AA2762177307840738F09F5F5F4F220F00
:106C4000331F441FAA1FA9F335D00E2E3AF0E0E8F7
:106C500032D091505040E695001CCAF72BD0FE2F41
:106C600029D0660F771F881FBB1F261737074807D5
:106C7000AB07B0E809F0BB0B802DBF01FF2793588D
:106C80005F4F3AF09E3F510578F00C94D5340C9448
:106C900020355F3FE4F3983ED4F38695779567956A
:106CA000B795F7959F5FC9F7880F911D96958795C2
:106CB00097F90895E1E0660F771F881FBB1F6217E1
:106CC00073078407BA0720F0621B730B840BBA0B9F
:106CD000EE1F88F7E09508950E9473366894B1110D
:106CE0000C94203508950E94053588F09F5798F040
:106CF000B92F9927B751B0F0E1F0660F771F881FC1
:106D0000991F1AF0BA95C9F714C0B13091F00E94DA
:106D10001F35B1E008950C941F35672F782F882711
:106D2000B85F39F0B93FCCF3869577956795B39501
:106D3000D9F73EF490958095709561957F4F8F4F70
:106D40009F4F08950E94413408F48FEF08950E94E8
:106D50004134880B990B0895AA1BBB1B51E107C056
:106D6000AA1FBB1FA617B70710F0A61BB70B881FDB
:106D7000991F5A95A9F780959095BC01CD0108956A
:106D800097FB072E16F4009407D077FD09D00E94D8
:106D9000AC3607FC05D03EF4909581959F4F089541
:106DA000709561957F4F0895A1E21A2EAA1BBB1B17
:106DB000FD010DC0AA1FBB1FEE1FFF1FA217B307C7
:106DC000E407F50720F0A21BB30BE40BF50B661FDD
:106DD000771F881F991F1A9469F7609570958095A1
:106DE00090959B01AC01BD01CF010895052E97FB45
:106DF0001EF400940E940D3757FD07D00E94D43630
:106E000007FC03D04EF40C940D3750954095309507
:106E100021953F4F4F4F5F4F089590958095709506
:106E200061957F4F8F4F9F4F0895EE0FFF1F059085
:106E3000F491E02D09940F931F93CF93DF93823049
:106E4000910510F482E090E0E091BF06F091C00659
:106E500030E020E0B0E0A0E0309799F42115310552
:106E600009F44AC0281B390B24303105D8F58A8132
:106E70009B816115710589F1FB0193838283FE017A
:106E800011C0408151810281138148175907E0F0F8
:106E90004817590799F4109761F012960C931297BE
:106EA00013961C933296CF01DF91CF911F910F91D2
:106EB00008950093BF061093C006F4CF2115310545
:106EC00051F04217530738F0A901DB019A01BD01C7
:106ED000DF01F801C1CFEF01F9CF9093C006809395
:106EE000BF06CDCFFE01E20FF31F81939193225095
:106EF000310939832883D7CF2091BD063091BE0652
:106F0000232B41F420912301309124013093BE06BC
:106F10002093BD06209121013091220121153105D8
:106F200041F42DB73EB74091250150912601241B15
:106F3000350BE091BD06F091BE06E217F307A0F411
:106F40002E1B3F0B2817390778F0AC014E5F5F4FBF
:106F50002417350748F04E0F5F1F5093BE0640932D
:106F6000BD06819391939FCFF0E0E0E09CCFCF935B
:106F7000DF930097E9F0FC01329713821282A0910F
:106F8000BF06B091C006ED0130E020E01097A1F4FB
:106F900020813181820F931F2091BD063091BE0662
:106FA0002817390709F061C0F093BE06E093BD06CB
:106FB000DF91CF910895EA01CE17DF07E8F54A8106
:106FC0005B819E0141155105B1F7E901FB83EA831D
:106FD00049915991C40FD51FEC17FD0761F48081C9
:106FE00091810296840F951FE9019983888382819C
:106FF00093819B838A83F0E0E0E012968D919C91CF
:1070000013970097B9F52D913C911197CD010296F8
:10701000820F931F2091BD063091BE0628173907B5
:1070200039F6309751F51092C0061092BF06B09312
:10703000BE06A093BD06BCCFD383C28340815181DD
:10704000840F951FC817D90761F44E5F5F4F888181
:107050009981480F591F518340838A819B81938373
:1070600082832115310509F0B0CFF093C006E0937B
:10707000BF069ECFFD01DC01C0CF13821282D7CFA5
:10708000B0E0A0E0E6E4F8E30C9449358C01009709
:1070900051F4CB010E941B378C01C801CDB7DEB77C
:1070A000E0E10C946535FC01E60FF71F9C012250CE
:1070B0003109E217F30708F49DC0D901CD91DC91A5
:1070C0001197C617D70798F0C530D10530F3CE0118
:1070D00004978617970708F3C61BD70B2297C1930F
:1070E000D1936D937C93CF010E94B737D6CF5B01CC
:1070F000AC1ABD0A4C018C0E9D1EA091BF06B0912A
:10710000C006512C412CF12CE12C109731F58091C7
:10711000BD069091BE068815990509F05CC046161B
:10712000570608F058C080912101909122010097E4
:1071300041F48DB79EB74091250150912601841BE3
:10714000950BE817F90708F055C0F093BE06E093D9
:10715000BD06F90171836083A0CF8D919C91119739
:1071600012966C90129713967C901397A815B905F8
:1071700059F56C0142E0C40ED11CCA14DB0420F1A5
:10718000AC014A195B09DA011296159780F0628208
:10719000738251834083D9016D937C93E114F10490
:1071A00071F0D7011396FC93EE93129776CF229647
:1071B0008C0F9D1FF90191838083F301EFCFF09332
:1071C000C006E093BF0669CF4816590608F42C01A3
:1071D0007D01D3019ACFCB010E941B377C01009720
:1071E00049F0AE01B8010E940539C8010E94B737C5
:1071F000870153CF10E000E050CF911108958156E0
:107200008A5108F4805285580895FB01DC0102C0C0
:1072100001900D9241505040D8F70895FB01DC01D8
:1072200001900D920020E1F70895FB01DC0141502F
:10723000504030F08D910190801919F40020B9F779
:10724000881B990B0895FB01DC014150504048F028
:1072500001900D920020C9F701C01D92415050408D
:10726000E0F70895FB0151915523A9F0BF01DC011E
:107270004D9145174111E1F759F4CD0101900020DE
:1072800049F04D9140154111C9F3FB014111EFCF78
:1072900081E090E00197089513E0C0E3D3E004C0DB
:1072A000FE010E9415372196C133D107C9F7F89422
:1072B000FFCF08200000008046030000A040C80067
:1072C00001CE0A0000000064000000F041F70E004B
:1072D00001200E0000C1068000FF018600000000B2
:1072E0000079000100FF0100FF005E00BC00770193
:1072F0000000000058049F03E503A5041604F403EE
:107300000804000000009F0A720ACC1147086B0AAB
:10731000580A490A0000000048089F03CC1147089A
:10732000A408BC082F0800000000A5119F03CC1181
:107330009E030D0A00202020202020202020202035
:1073400020202000524542005645520023566572C7
:1073500073696F6E3A004C4F4700234C6F67676547
:1073600072204E616D653A0053484F57533D0047B8
:10737000455400732000534156453D0054494D4546
:10738000493D0023496E74657276616C3D00544935
:107390004D45443D00234475726174696F6E3D0034
:1073A00042543D00534C20503D00506120756E6C9E
:1073B000696B656C792100685061004E45543D0051
:1073C00055565A002355562056303D00562000444D
:1073D000535400234453542063616C696272617496
:1073E000656420666F722023004D533D002C0023FE
:1073F000496E636F727265637421204D533D313263
:107400003344334435005428312C322C33293D0089
:10741000445354286F432900206F43204453205481
:107420006865726D6F6D657465720020572F6D5EB3
:107430003200555620496E74656E73697479005731
:107440002F6D5E32200055563D0070706D00434F29
:107450003220436F6E632E00434F323D004C69670C
:10746000687420496E74656E7369747900206C7855
:1074700020004C3D00495220466C616D65204C65F2
:1074800076656C3D00476173206C6576656C3D00E8
:10749000204D756C746973656E736F72730023454C
:1074A0006E61626C65002344697361626C650044BF
:1074B000440023496E76616C6964206B6579210014
:1074C000424E4D4C3033004244326936445354638B
:1074D00000234E6F2053656E736F72210057656CE9
:1074E000636F6D653A0073657269616C3A20002DB7
:0874F00035002D34002D33009E
:107E0000112484B714BE81FFF0D085E080938100F7
:107E100082E08093C00088E18093C10086E0809377
:107E2000C20080E18093C4008EE0C9D0259A86E02C
:107E300020E33CEF91E0309385002093840096BBD3
:107E4000B09BFECF1D9AA8958150A9F7CC24DD24C4
:107E500088248394B5E0AB2EA1E19A2EF3E0BF2EE7
:107E6000A2D0813461F49FD0082FAFD0023811F036
:107E7000013811F484E001C083E08DD089C08234E0
:107E800011F484E103C0853419F485E0A6D080C0E4
:107E9000853579F488D0E82EFF2485D0082F10E0AE
:107EA000102F00270E291F29000F111F8ED06801E7
:107EB0006FC0863521F484E090D080E0DECF843638
:107EC00009F040C070D06FD0082F6DD080E0C81688
:107ED00080E7D80618F4F601B7BEE895C0E0D1E017
:107EE00062D089930C17E1F7F0E0CF16F0E7DF06D8
:107EF00018F0F601B7BEE89568D007B600FCFDCFD4
:107F0000A601A0E0B1E02C9130E011968C91119780
:107F100090E0982F8827822B932B1296FA010C0160
:107F200087BEE89511244E5F5F4FF1E0A038BF0790
:107F300051F7F601A7BEE89507B600FCFDCF97BE46
:107F4000E89526C08437B1F42ED02DD0F82E2BD052
:107F50003CD0F601EF2C8F010F5F1F4F84911BD097
:107F6000EA94F801C1F70894C11CD11CFA94CF0C13
:107F7000D11C0EC0853739F428D08EE10CD085E9AC
:107F80000AD08FE07ACF813511F488E018D01DD067
:107F900080E101D065CF982F8091C00085FFFCCF94
:107FA0009093C60008958091C00087FFFCCF809118
:107FB000C00084FD01C0A8958091C6000895E0E648
:107FC000F0E098E1908380830895EDDF803219F02E
:107FD00088E0F5DFFFCF84E1DECF1F93182FE3DFCA
:107FE0001150E9F7F2DF1F91089580E0E8DFEE27F6
:047FF000FF270994CA
:027FFE00040479
:00000001FF
